:020000040800F2
:100000000080012007680008516700087D6800082B
:10001000556700085767000859670008000000008E
:100020000000000000000000000000005B67000806
:100030005D670008000000005F670008BD29000838
:10004000636700086567000867670008696700085C
:100050006B6700086D6700086F670008716700082C
:1000600073670008756700087767000879670008FC
:100070007B6700087D6700087F67000881670008CC
:10008000836700088567000887670008896700089C
:100090008B6700088D6700088F670008916700086C
:1000A000936700089567000897670008996700083C
:1000B0009B6700089D6700089F670008A16700080C
:1000C000A3670008A5670008A7670008A9670008DC
:1000D000AB670008C12A0008092B0008B1670008B7
:1000E000B3670008B5670008B7670008B96700087C
:1000F000BB670008BD670008BF670008C16700084C
:10010000C3670008C5670008C7670008C96700081B
:10011000CB670008CD670008CF670008D1670008EB
:10012000D3670008D5670008D7670008D9670008BB
:10013000DB670008DD670008DF670008E16700088B
:10014000E3670008E5670008E767000845750008F1
:10015000EB670008ED670008EF670008F16700082B
:10016000F3670008F5670008F7670008F9670008FB
:10017000FB670008FD670008FF67000801680008CA
:0801800003680008056800088F
:1001880082B003468DF807309DF90730002B0CDB51
:100198009DF8073003F01F0205499DF907305B09F8
:1001A800012000FA02F241F8232000BF02B0704794
:0401B80000E100E082
:1001BC0082B0034600918DF807309DF90730002B73
:1001CC000ADB009BDAB20C499DF907301201D2B25E
:1001DC000B4483F800230BE0009BDAB207499DF82F
:1001EC00073003F00F03043B1201D2B20B441A7612
:1001FC0000BF02B0704700BF00E100E000ED00E07E
:10020C0000B583B00190019B013BB3F1807F01D31A
:10021C0001230FE0094A019B013B53600F214FF072
:10022C00FF30FFF7C5FF054B00229A60034B0722F6
:10023C001A600023184603B05DF804FB10E000E0E0
:10024C0000B583B0854B9B6D844A43F08053936516
:10025C00824BDB6C814A43F00103D3647F4BDB6C34
:10026C007E4A43F00203D3647C4BDB6C7B4A43F045
:10027C000403D364794BDB6C784A43F00803D364F2
:10028C004FF0904300221A60754B00221A60754B98
:10029C0000221A60744B00221A604FF09043734A8C
:1002AC00DA606F4B724ADA606E4B724ADA606E4BF0
:1002BC002022DA6000F0A2FC4FF090431B684FF054
:1002CC00904223F002031360664B1B68654A43F0AF
:1002DC0001031360634B1B68624A43F00403136011
:1002EC00604B03229A614FF090431B684FF0904291
:1002FC0023F4006313604FF090431B684FF090425F
:10030C0043F4806313605C4B1B685C4AA2FB0323C1
:10031C009B091846FFF774FF594B14221A60594B6E
:10032C0000221A60584B00221A60584B00221A60A7
:10033C00574B00221A60574B4FF47A721A60564B87
:10034C004FF47A721A60554B00221A60544B0022FB
:10035C001A60544B00221A60534B00221A60534B04
:10036C0001221A60524B00221A60524B00221A6072
:10037C00514B00221A60514B00221A60504B45F22F
:10038C0055521A604E4B4FF6FF729A60022000F0E5
:10039C00D3FC4B4B02225A60022000F0CDFC484BA0
:1003AC004CF6CC421A602F4BDB682E4A43F05003BC
:1003BC00D3602C4BDB682B4A23F0A003D3600220C4
:1003CC0000F0BAFC3F4B00221A60264B1B6903F06D
:1003DC000403002B02D13B4B01221A6001F066FC96
:1003EC0001F08AFF02F0ECF8364B1B68002B14D19D
:1003FC000A2000F0A1FC4F2002F0CCF86B2002F098
:10040C00C9F80D2002F0C6F84F2002F029F96B2034
:10041C0002F026F90D2002F023F90A2000F08CFCE2
:10042C00294B00221A6002F0F3FB194B40F6B8324C
:10043C001A6003E0164B1B68002B04D0224B1B6880
:10044C00002BF7D000E000BF06F07FFC184B002219
:10045C001A6000238DF8053043E000BF0010024005
:10046C000004004800080048000C0048AAAA02A496
:10047C008AAAAAAAAAAAAAA610000020D34D621082
:10048C00844100209841002088410020A841002090
:10049C007841002094410020604100207C410020E4
:1004AC004C410020804100209C41002090410020C4
:1004BC00A0410020A4410020744100208C41002068
:1004CC000030004044410020484100209DF8053098
:1004DC00934A002122F813109DF8053001338DF852
:1004EC0005309DF80530112BF0D901F051F864203E
:1004FC0000F022FC00F0D4FC642000F01DFC00F0A5
:10050C00CFFC0A2000F018FC864B00221A60864BA8
:10051C001B6903F00803002B02D1824BFF221A60E7
:10052C000A2000F009FC814B1B68002B05D1804B85
:10053C001B68002B01D004F0D1F802F08FF90346B0
:10054C00ADF80630BDF80630002B04D102F0C2F92C
:10055C000346ADF80630BDF80630002B64D0BDF86C
:10056C0006308DF80530714B1B68002B57D1714B41
:10057C001B68002B4DD1704B1B68042B06D16F4BA5
:10058C001B68002B02D06C4B00221A609DF80530C2
:10059C002B2B0AD1684B1B68022B06D1664B03220E
:1005AC001A60664B4FF47A721A609DF805302B2B4B
:1005BC000AD1614B1B68012B06D15F4B02221A60DA
:1005CC005E4B4FF4C8721A609DF805302B2B0ED180
:1005DC00594B1B68002B0AD1584B1B68002B06D1BA
:1005EC00554B01221A60554B4FF4C8721A60504B90
:1005FC001B68002B18D19DF80530184603F0F6FD4A
:10060C004D4B1B68002B0FD14C4B4FF47A721A6078
:10061C000AE09DF80530184603F0E8FD04E09DF86B
:10062C000530184603F008FE454B1B68002B3FF4C1
:10063C007AAF03F035FC0346ADF80630BDF8063052
:10064C00002B3FF470AFBDF806308DF80530374BFA
:10065C001B68002B59D1384B1B68002B7FF463AF00
:10066C00344B1B68042B06D1364B1B68002B02D075
:10067C00304B00221A609DF805302B2B0AD12D4BE4
:10068C001B68022B06D12B4B03221A602D4B4FF407
:10069C007A721A609DF805302B2B0AD1254B1B68FA
:1006AC00012B06D1234B02221A60264B4FF4C87241
:1006BC001A609DF805302B2B0ED11E4B1B68002B9E
:1006CC000AD1204B1B68002B06D11A4B01221A6051
:1006DC001C4B4FF4C8721A60154B1B68002B7FF42F
:1006EC0022AF9DF80530184601F054FF9DF80530F7
:1006FC00184601F0B5FF0F4B1B68002B7FF413AFAE
:10070C00104B4FF47A721A600DE79DF805301846BD
:10071C0001F040FF9DF80530184601F0A1FF02E7FB
:10072C00E8400020A041002000080048444100207F
:10073C00804100204C4100207C410020944100204D
:08074C0048410020604100203B
:1007540082B00190019B033B0E2B00F23A8201A26E
:1007640052F823F0A5070008FB07000869080008F1
:10077400D708000845090008770900089D09000802
:10078400C3090008E9090008190A0008870A0008D3
:10079400F70A0008650B00088B0B0008B10B000872
:1007A4009A4B1B68994A23F003031360974BDB6849
:1007B400964A23F00203D360944BDB68934A43F0D8
:1007C4000103D360924B5B8B1BB2002B80F203823C
:1007D4008E4B1B688D4A43F0030313608B4BDB681D
:1007E4008A4A23F00303D360884BDB6A874A43F0C9
:1007F4000103D362EFE14FF090431B684FF0904246
:1008040023F4407313604FF09043DB684FF0904241
:1008140023F40073D3604FF09043DB684FF09042B1
:1008240043F48073D3607A4BDB8B1BB2002B80F2D2
:10083400D4814FF090431B684FF0904243F44073CF
:1008440013604FF09043DB684FF0904223F4407301
:10085400D3604FF09043DB6A4FF0904243F01003B3
:10086400D362BAE14FF090431B684FF0904223F0FB
:100874000C0313604FF09043DB684FF0904223F079
:100884000803D3604FF09043DB684FF0904243F08D
:100894000403D3605E4B5B8C1BB2002B80F29F8100
:1008A4004FF090431B684FF0904243F00C031360E9
:1008B4004FF09043DB684FF0904223F00C03D36079
:1008C4004FF09043DB6A4FF0904243F00203D3624F
:1008D40085E14FF090431B684FF0904223F00303EF
:1008E40013604FF09043DB684FF0904223F0020313
:1008F400D3604FF09043DB684FF0904243F0010324
:10090400D360434BDB8C1BB2002B80F26A814FF027
:1009140090431B684FF0904243F0030313604FF081
:100924009043DB684FF0904223F00303D3604FF011
:100934009043DB6A4FF0904243F00103D36250E1ED
:100944004FF090431B684FF0904223F040431360F4
:100954004FF09043DB684FF0904223F00043D360A4
:100964004FF09043DB684FF0904243F08043D360F4
:100974003EE1264B1B68254A23F440431360234B76
:10098400DB68224A23F40043D360204BDB681F4A10
:1009940043F48043D3602BE11C4B1B681B4A23F0B8
:1009A400C0031360194BDB68184A23F0C003D360FB
:1009B400164BDB68154A43F04003D36018E1134B30
:1009C4001B68124A23F440631360104BDB680F4A20
:1009D40023F44063D3600D4BDB680C4A43F480631B
:1009E400D36005E1094B1B68084A23F44073136084
:1009F400064BDB68054A23F44073D360034BDB6882
:100A0400024A43F48073D360F2E000BF000400485C
:100A14006C4000204FF090431B684FF0904223F449
:100A2400404313604FF09043DB684FF0904223F44F
:100A34000043D3604FF09043DB684FF0904243F49F
:100A44008043D3606C4BDB8F1BB2002B80F2CB80D6
:100A54004FF090431B684FF0904243F440431360BF
:100A64004FF09043DB684FF0904223F44043D3604F
:100A74004FF09043DB6A4FF0904243F08003D3621F
:100A8400B1E04FF090431B684FF0904223F4405381
:100A940013604FF09043DB684FF0904223F400530F
:100AA400D3604FF09043DB684FF0904243F480539F
:100AB400D360514BB3F842301BB2002B80F29580C7
:100AC4004FF090431B684FF0904243F4405313603F
:100AD4004FF09043DB684FF0904223F44053D360CF
:100AE4004FF09043DB6A4FF0904243F04003D362EF
:100AF4007BE04FF090431B684FF0904223F4406337
:100B040013604FF09043DB684FF0904223F400638E
:100B1400D3604FF09043DB684FF0904243F480631E
:100B2400D360354BB3F846301BB2002B5FDA4FF07D
:100B340090431B684FF0904243F4406313604FF0BE
:100B44009043DB684FF0904223F44063D3604FF04E
:100B54009043DB6A4FF0904243F02003D36246E0B7
:100B6400264B1B68254A23F440231360234BDB6880
:100B7400224A23F44023D360204BDB681F4A43F40A
:100B84008023D36034E01D4B1B681C4A23F440339C
:100B940013601A4BDB68194A23F44033D360174BB4
:100BA400DB68164A43F48033D36021E0144B1B689E
:100BB400134A23F040631360114BDB68104A23F09F
:100BC4004063D3600E4BDB680D4A43F08063D3600F
:100BD4000EE000BF0CE000BF0AE000BF08E000BF69
:100BE40006E000BF04E000BF02E000BF00E000BF79
:100BF40000BF02B0704700BF6C40002000040048F2
:040C0400000800489C
:100C0800424B9B6D414A43F08053936500BF404B74
:100C18005B6903F48063002BF9D13D4B1B683C4AA8
:100C280023F4806313603A4B1B68394A43F44073DA
:100C3800136000BF364B5B6903F48063002BF9D166
:100C4800344B1B68334A43F4817313602F4B1B6882
:100C58002E4A23F08073136000BF2C4B1B6803F0EF
:100C68000073002BF9D1294BD3F89030274A23F091
:100C78003D03C2F89030254BD3F89030234A43F017
:100C88001803C2F89030214BD3F890301F4A43F034
:100C98000103C2F8903000BF1C4BD3F8903003F02A
:100CA8000203002BF8D000BF184B1B6803F00203A7
:100CB800002BF9D0154B1B68144A23F0F00313607E
:100CC800124B1B68114A43F0B00313600F4B1B68AB
:100CD8000E4A43F00D03136000BF0C4B1B6803F072
:100CE8000203002BF9D0094B9B68084A43F41053C0
:100CF8009360064BD3F88830044A43F04063C2F847
:100D08008830054B054A1A6000BF70470010024042
:100D1800007000400020024010000020006CDC023F
:100D2800044B4FF400329A61034BC8221A6000BF8B
:0C0D3800704700BF000800488841002000
:100D440082B00346ADF80630BDF80630054A13609C
:100D540000BF044B1B68002BFBD100BF00BF02B0D7
:080D6400704700BFA841002008
:100D6C0008B5444B14221A60434B4AF6AA221A6067
:100D7C00424B1B68002B01D100F092F8404B1B68D2
:100D8C00002B02D13F4B01229A613F4B1B68002B79
:100D9C0002D13C4B02229A613C4B1B6801333B4A0B
:100DAC0013603A4B1B68312B62D9384B00221A6006
:100DBC00374B9B884FF6FF72934203D1354B002281
:100DCC001A7004E0324B9B88DAB2324B1A702D4BFE
:100DDC001B6903F00403002B11D12F4B1B68002B54
:100DEC000DD101F0EBFE2C4B01221A6001F084FABC
:100DFC004FF4FA70FFF7A0FF01F00AFF16E0214B49
:100E0C001B6903F00403002B10D0234B1B68012B30
:100E1C000CD101F0D3FE204B00221A6001F06CFAC9
:100E2C004FF4FA70FFF788FF01F0F2FE134B1B68CA
:100E3C00002B1AD1134B1B6903F00803002B06D1AE
:100E4C00164B1B68002B02D1144BFF221A600D4B62
:100E5C001B6903F00803002B0AD0104B1B68002BF6
:100E6C0006D00E4B00221A6002E00C4B00221A60D6
:100E7C0000BF08BD8441002000300040A441002088
:100E8C00984100200008004888410020344100208F
:100E9C0014400020C641002044410020A041002005
:100EAC0000B583B0AC4B9B6803F00103002B01D160
:100EBC0000F06EFBA94B5B8B4FF6FF72934222D076
:100ECC00A64B5B8B1BB2002B10DAA54B1B68002BBF
:100EDC000CD00F2000F00AFB0346ADF80630BDF82D
:100EEC0006301946032000F0C1F90CE09D4B1B693C
:100EFC009BB203F00103ADF80430BDF80430194681
:100F0C00032000F0B5FA954BDB8B4FF6FF72934242
:100F1C0023D0924BDB8B1BB2002B10DA904B1B684F
:100F2C00002B0CD0092000F0E1FA0346ADF8063096
:100F3C00BDF806301946042000F098F90DE04FF08A
:100F4C0090431B699BB203F01003ADF80430BDF85D
:100F5C0004301946042000F08BFA804B5B8C4FF662
:100F6C00FF72934223D07D4B5B8C1BB2002B10DAAB
:100F7C007B4B1B68002B0CD0062000F0B7FA034605
:100F8C00ADF80630BDF806301946052000F06EF9B4
:100F9C000DE04FF090431B699BB203F00203ADF8D8
:100FAC000430BDF804301946052000F061FA6B4B93
:100FBC00DB8C4FF6FF72934223D0684BDB8C1BB259
:100FCC00002B10DA664B1B68002B0CD0052000F0B0
:100FDC008DFA0346ADF80630BDF8063019460620EA
:100FEC0000F044F90DE04FF090431B699BB203F005
:100FFC000103ADF80430BDF804301946062000F0AA
:10100C0037FA564B5B8D4FF6FF7293420FD04FF071
:10101C0090431B699BB223F4FF4323F07F03ADF88D
:10102C000430BDF804301946072000F021FA4B4B70
:10103C00DB8D4FF6FF7293420CD04A4B1B699BB26F
:10104C0003F08003ADF80430BDF8043019460820D5
:10105C0000F00EFA414B5B8E4FF6FF7293420CD0B0
:10106C00404B1B699BB203F00803ADF80430BDF88C
:10107C0004301946092000F0FBF9384BDB8E4FF693
:10108C00FF7293420CD0374B1B699BB203F02003C9
:10109C00ADF80430BDF8043019460A2000F0E8F928
:1010AC002E4B5B8F4FF6FF7293420CD02D4B1B696E
:1010BC009BB203F01003ADF80430BDF804301946B0
:1010CC000B2000F0D5F9254BDB8F4FF6FF729342C6
:1010DC0023D0224BDB8F1BB2002B10DA204B1B686A
:1010EC00002B0CD00C2000F001FA0346ADF80630B2
:1010FC00BDF8063019460C2000F0B8F80DE04FF0A2
:10110C0090431B699BB203F08003ADF80430BDF82B
:10111C00043019460C2000F0ABF9104BB3F84230F8
:10112C004FF6FF7293422DD00C4BB3F842301BB2EA
:10113C00002B19DA0A4B1B68002B15D00B2000F082
:10114C00D5F90346ADF80630BDF8063019460D202A
:10115C0000F08CF816E000BF000004506C4000203A
:10116C00AC410020000400484FF090431B699BB237
:10117C0003F04003ADF80430BDF8043019460D20DF
:10118C0000F076F9354BB3F846304FF6FF729342C8
:10119C0024D0324BB3F846301BB2002B10DA304B54
:1011AC001B68002B0CD00A2000F0A0F90346ADF808
:1011BC000630BDF8063019460E2000F057F80DE049
:1011CC004FF090431B699BB203F02003ADF8043041
:1011DC00BDF8043019460E2000F04AF91F4BB3F845
:1011EC004A304FF6FF7293420CD01E4B1B699BB2D8
:1011FC0003F40073ADF80430BDF8043019460F2029
:10120C0000F036F9154BB3F84E304FF6FF7293429F
:10121C000CD0144B1B699BB203F48073ADF80430F3
:10122C00BDF804301946102000F022F90B4BB3F82E
:10123C0052304FF6FF7293420CD00B4B1B699BB292
:10124C0003F40053ADF80430BDF8043019461120F6
:10125C0000F00EF900BF03B05DF804FB6C400020F9
:0C126C00AC4100200004004800080048CD
:1012780000B585B003460A468DF807301346ADF829
:1012880004309DF807305B005B00744A13440293F6
:10129800029B1B884FF6FF72934200F0D980029B95
:1012A80002331B884FF6FF72934200F0D3806C4BD9
:1012B800DB88ADF80E30029B1B88ADF80C30BDF80A
:1012C8000C3003F0F003002B04D0BDF80C301B09E0
:1012D800ADF80C30BDF80C300E2B07D1029B023351
:1012E8001B8803F47F43B3F5014F0DD0BDF80430DC
:1012F8005B09ADF80430BDF80E30002B04D0BDF802
:101308000E30023BADF80E309DF80730554A32F8E2
:101318001330BDF804209A4200F09D809DF80730F4
:10132800514AD35C002B49D09DF807304D4A32F81A
:101338001330BDF804209A4216D29DF807304B4965
:10134800BDF8042021F81320494B1B68002B04D05A
:101358009DF80730184600F081F99DF8073041499B
:10136800BDF8042021F81320BDF804209DF80730AB
:101378003C4931F813301946BDF80E300B449A42F7
:1013880069DD9DF807303949BDF8042021F813209C
:10139800374B1B68002B04D09DF80730184600F027
:1013A8005DF99DF807302F49BDF8042021F8132076
:1013B8009DF807302C4A0021D1544CE09DF80730A5
:1013C800284A32F81330BDF804209A4216D99DF8FD
:1013D80007302649BDF8042021F81320244B1B6848
:1013E800002B04D09DF80730184600F037F99DF817
:1013F80007301C49BDF8042021F81320BDF804204B
:101408009DF80730174931F813301946BDF80E30EA
:10141800CB1A9A421FDA9DF807301449BDF8042008
:1014280021F81320124B1B68002B04D09DF80730BD
:10143800184600F013F99DF807300A49BDF8042052
:1014480021F813209DF80730074AFF21D15402E004
:1014580000BF00E000BF05B05DF804FB204000209D
:1014680014400020C440002020410020E840002013
:04147800A04100206F
:10147C0000B583B003460A468DF807301346ADF825
:10148C0004309DF80730164A32F81330BDF80420AA
:10149C009A4207D09DF807301149BDF8042021F875
:1014AC00132018E09DF807300E4A32F81330BDF8BF
:1014BC0004209A420FD09DF807300A49BDF8042049
:1014CC0021F81320084B1B68002B04D09DF8073023
:1014DC00184600F0D9F900BF03B05DF804FB00BF5B
:0C14EC00C4400020E8400020A041002087
:1014F80086B003468DF807300023059300238DF846
:1015080013301FE0224B40F2FF721A609DF807303B
:101518009A011F4B1A631E4B9B681D4A43F0040334
:10152800936000BF1A4B1B6803F00403002BF9D02B
:10153800174B1B6C059A134405939DF81330013320
:101548008DF813309DF81330412BDBD9059B03F040
:101558000F030393059B1B090593039B072B02D9D4
:10156800059B01330593059B403B0593059BB3F110
:101578007F4F01D900230593059BB3F5805F02D304
:1015880040F6FF730593059B9BB2184606B070475B
:0415980000000450FB
:10159C0008B52B4BDB6C2A4A43F40053D364294B1C
:1015AC009B68284A23F000539360264B9B68254A7E
:1015BC0043F0805393600220FFF7BEFB214BD3F81E
:1015CC00B030204A1B0C1B04C2F8B0301E4B4FF439
:1015DC0000329A600220FFF7AFFB1A4B1B68194AC6
:1015EC0043F001031360174B9B68164A43F0010349
:1015FC00936000BF134B1B6803F00103002BF9D061
:10160C00104B1B680F4A43F0010313600D4B08226B
:10161C00DA600C4B0D4A5A610A4B0D4A9A61094B20
:10162C0000221A63074B00225A63064B00229A636E
:10163C00044B0022DA63074BFF221A6000BF08BD7F
:10164C0000100240000004500003045000806D1B89
:08165C00DB800100AC4100201D
:1016640000B587B003468DF807309DF807305B005E
:101674005B00834A13440393039B1B884FF6FF725A
:10168400934200F0F580039B1B88DBB2ADF80A306F
:10169400BDF80A30F32B00F2ED80BDF80A308DF866
:1016A40017309DF817300F2B0AD89DF817301B01FF
:1016B4005AB2744B1B785BB213435BB28DF817308C
:1016C4009DF817301B09DBB2ADF80A30039B0233D7
:1016D4000393039B1B88ADF80830BDF808304FF620
:1016E400FF72934200F0C880674B1B68012B04D142
:1016F4009DF81730184605F045FE9DF80730634AFB
:1017040032F81330ADF81230BDF80A300E2B44D144
:10171400BDF8083003F47F43B3F5014F17D1BDF88A
:101724001230DBB29B00DBB203F07C038DF8163081
:10173400BDF812305B099BB28DF81530BDF812303C
:101744006FEA43436FEA5343ADF8123009E00023D4
:101754008DF81630BDF81230DBB203F07F038DF83C
:101764001530494B1B68012B0DD19DF816301846D6
:1017740005F008FE9DF8153003F07F03DBB2184630
:1017840005F000FE79E0BDF812209DF807109DF8E1
:101794001730184600F064F96FE0BDF80A300B2BDF
:1017A40003D99DF81730F22B27D1039B1B88DBB29A
:1017B40003F07F038DF81630BDF81230DBB203F06E
:1017C4007F038DF81530304B1B68012B0AD19DF82F
:1017D4001630184605F0D6FD9DF81530184605F06C
:1017E400D1FD4AE09DF815309AB29DF807109DF896
:1017F4001730184600F034F93FE0BDF80A300C2BDE
:1018040007D0BDF80A300D2B03D09DF81730F32B09
:101814001BD1BDF81230DBB203F07F038DF8153015
:10182400194B1B68012B05D19DF81530184605F09E
:10183400A9FD22E09DF815309AB29DF807109DF895
:101844001730184600F00CF917E00F4B1B68012BFA
:1018540006D1002005F096FD002005F093FD0CE074
:101864009DF8173000221946452000F0F9F804E0ED
:1018740000BF02E000BF00E000BF07B05DF804FB5A
:1018840020400020C641002044410020E8400020C0
:1018940000B587B003468DF807309DF807305B002C
:1018A4005B006B4A13440493049B9A1C04921B88A8
:1018B400DBB2ADF80E30BDF80E30F52B23D9BDF8F0
:1018C4000E30F92B1FD0BDF80E30FD2B1BD09DF828
:1018D4000730604A32F81330002B40F0B5805E4B7D
:1018E4001B68012B06D1BDF80E30DBB2184605F09B
:1018F40049FDA9E0BDF80E209DF8073019460020E7
:1019040000F0AEF8A0E0BDF80E308DF817309DF869
:1019140017300F2B0AD89DF817301B015AB24F4BC2
:101924001B785BB213435BB28DF817304A4B1B68CC
:10193400012B04D19DF81730184605F023FD9DF8BE
:1019440017301B09DBB2ADF80E30BDF80E300E2B8C
:1019540003D100238DF8163006E0049B1B88DBB20C
:1019640003F07F038DF816309DF80730394A32F8BA
:101974001330002B03D000238DF8153008E0049BAE
:101984001B881B0A9BB2DBB203F07F038DF8153072
:10199400BDF80E300C2B07D0BDF80E300D2B03D044
:1019A4009DF81730F32B13D12B4B1B68012B05D15A
:1019B4009DF81530184605F0E5FC46E09DF8153015
:1019C4009AB29DF807301946002000F049F83CE02F
:1019D400BDF80E30082B03D9BDF80E300B2B07D9F8
:1019E400BDF80E300E2B03D09DF81730F22B18D112
:1019F400194B1B68012B0AD19DF81630184605F0C7
:101A0400C1FC9DF81530184605F0BCFC1DE09DF89E
:101A140015309AB29DF807301946002000F020F8DE
:101A240013E00D4B1B68012B06D1002005F0AAFC26
:101A3400002005F0A7FC08E09DF8173000221946A5
:101A4400452000F00DF800E000BF07B05DF804FB8E
:101A540020400020E840002044410020C6410020EE
:101A640000B585B003468DF807300B468DF8063077
:101A74001346ADF804308D4A02AB92E803001860B7
:101A84000433198002330A0C1A70202000F002FE7D
:101A94009DF80730002B48D1232000F0FBFD9DF872
:101AA4000630112B03D1752000F0F4FD15E09DF8EC
:101AB4000630092B0AD9312000F0ECFD9DF80630E0
:101AC4002633DBB2184600F0E5FD06E09DF806304B
:101AD4003033DBB2184600F0DDFD642000F0DAFD9F
:101AE400BDF80430002B03D1302000F0D3FDD5E045
:101AF4006F4B1B68002B0FD0302000F0CBFD7820FB
:101B040000F0C8FDBDF80430DBB203F07F03DBB2A4
:101B1400184605F05CF9C1E0BDF8043003F07F031A
:101B24009BB2184600F018FEB8E09DF80730452B2C
:101B34002ED102AB184605F0EBFC232000F0AAFDE1
:101B44009DF80630112B03D1752000F0A3FD15E09C
:101B54009DF80630092B0AD9312000F09BFD9DF831
:101B640006302633DBB2184600F094FD06E09DF8FB
:101B740006303033DBB2184600F08CFD452000F00F
:101B840089FD722000F086FD722000F083FD85E05F
:101B9400232000F07FFD9DF80630112B03D1752022
:101BA40000F078FD15E09DF80630092B0AD93120A4
:101BB40000F070FD9DF806302633DBB2184600F0C5
:101BC40069FD06E09DF806303033DBB2184600F0BC
:101BD40061FD612000F05EFD9DF8073003F0F00325
:101BE400E02B3FD1BDF90430002B1EDA682000F051
:101BF40051FD2F4B1B68002B0ED0302000F04AFD06
:101C0400782000F047FDBDF80430C3F30B039BB20A
:101C1400184605F022F941E0BDF80430C3F30B0384
:101C24009BB2184600F098FD38E0214B1B68002B4E
:101C34000FD0302000F02EFD782000F02BFDBDF8F1
:101C44000430DBB203F07F03DBB2184605F0BFF8C3
:101C540024E0BDF8043003F07F039BB2184600F083
:101C64007BFD1BE0124B1B68002B0FD0302000F0D3
:101C740011FD782000F00EFDBDF80430DBB203F056
:101C84007F03DBB2184605F0A2F807E0BDF8043084
:101C940003F07F039BB2184600F05EFD202000F0A5
:101CA400F9FC00BF05B05DF804FB00BF80730008B9
:041CB400904100203B
:101CB80000B585B0044B0293044B0193044B009389
:101CC80000238DF80F301BE0007800086C400020DE
:101CD80014400020029B1A88019B1A80029B1A88D4
:101CE800009B1A80019B02330193009B02330093EF
:101CF800029B023302939DF80F3001338DF80F30A9
:101D08009DF80F302B2BE5D9984B1B884FF6FF72A7
:101D1800934205D1954B0B221A80954B0B221A80C2
:101D2800924B5B884FF6FF72934205D18F4B1F226F
:101D38005A808F4B1F225A808C4B9B884FF6FF721C
:101D4800934205D1894B00229A80894B00229A80C0
:101D5800864BDB884FF6FF72934205D1834B0422F2
:101D6800DA80834B0422DA80804B1B894FF6FF729E
:101D7800934205D07D4B5B894FF6FF7293420BD19E
:101D88007A4B04221A81794B83225A81784B042298
:101D98001A81774B83225A81744B9B894FF6FF72C5
:101DA800934205D0714BDB894FF6FF7293420BD1FA
:101DB8006E4B57229A816D4B4022DA816C4B572229
:101DC8009A816B4B4022DA81684B1B8A4FF6FF726F
:101DD80093420ED1654B0B221A82644B1A8A644BCC
:101DE8001A82624B44F201025A82614B44F20102A8
:101DF8005A825E4B9B8A4FF6FF7293420ED15B4B21
:101E08000B229A82594B9A8A594B9A82574B44F221
:101E18000202DA82564B44F20202DA82534B1B8BDF
:101E28004FF6FF7293420ED1504B0B221A834F4B41
:101E38001A8B4F4B1A834D4B44F203025A834C4B77
:101E480044F203025A83494B9B8B4FF6FF7293422D
:101E58000ED1464B0B229A83444B9A8B444B9A8360
:101E6800424B44F20402DA83414B44F20402DA831F
:101E78003E4B1B8C4FF6FF7293420ED13B4B0E220A
:101E88001A843A4B1A8C3A4B1A84384B4FF4014255
:101E98005A84374B4FF401425A84344B9B8C4FF68B
:101EA800FF7293420ED1314B0B229A842F4B9A8C9E
:101EB8002F4B9A842D4B44F20602DA842C4B44F2C1
:101EC8000602DA84294B1B8D4FF6FF7293420ED11E
:101ED800264B0B221A85254B1A8D254B1A85234B29
:101EE80044F207025A85224B44F207025A851F4BD7
:101EF8009B8D4FF6FF7293420ED11C4B0B229A8595
:101F08001A4B9A8D1A4B9A85184B44F20802DA85B7
:101F1800174B44F20802DA85144B1B8E4FF6FF72FA
:101F280093420ED1114B0B221A86104B1A8E104B6E
:101F38001A860E4B44F209025A860D4B44F20902E6
:101F48005A860A4B9B8E4FF6FF72934213D1074B6A
:101F58000B229A86054B9A8E054B9A86034B44F2C0
:101F68000A02DA86024B44F20A0203E06C400020BF
:101F780014400020DA866A4B1B8F4FF6FF7293429B
:101F88000ED1674B0B221A87654B1A8F654B1A8740
:101F9800634B44F20B025A87624B44F20B025A8796
:101FA8005F4B9B8F4FF6FF7293420ED15C4B0B2217
:101FB8009A875B4B9A8F5B4B9A87594B44F20C027A
:101FC800DA87584B44F20C02DA87554BB3F84030A5
:101FD8004FF6FF72934213D1514B0E22A3F84020C3
:101FE8004F4BB3F840204F4BA3F840204C4B4FF4D5
:101FF8000042A3F842204B4B4FF40042A3F8422082
:10200800474BB3F844304FF6FF72934213D1444B19
:102018000B22A3F84420424BB3F84420414BA3F8C9
:1020280044203F4B44F20E02A3F846203D4B44F2B5
:102038000E02A3F846203A4BB3F848304FF6FF7229
:10204800934213D1364B0B22A3F84820344BB3F8F4
:102058004820344BA3F84820314B44F20F02A3F830
:102068004A20304B44F20F02A3F84A202C4BB3F815
:102078004C304FF6FF72934213D1294B0B22A3F831
:102088004C20274BB3F84C20264BA3F84C20244B6C
:1020980044F21002A3F84E20224B44F21002A3F897
:1020A8004E201F4BB3F850304FF6FF72934213D1B6
:1020B8001B4B0B22A3F85020194BB3F85020194B97
:1020C800A3F85020164B44F21102A3F85220154BE6
:1020D80044F21102A3F85220114BB3F854304FF6D2
:1020E800FF72934207D10E4B0122A3F854200D4BE7
:1020F8000122A3F854200A4B9B88DAB20A4B1A70C3
:10210800074BB3F854301A46084B1A60084B0022A4
:102118001A6004F01CFE00BF05B05DF804FB00BFA8
:102128006C40002014400020C6410020904100204F
:042138009C410020A6
:10213C0000B585B000BF684B1B6903F48033002BDE
:10214C00F9D1654B5B69002B05DA634B634A9A60E6
:10215C00614B634A9A6000BF5F4B1B6903F4803389
:10216C00002BF9D15C4B5F4A5A615B4B5B695A4A55
:10217C0043F48033536100BF574B1B6903F4803326
:10218C00002BF9D1544B1B6903F00103002B06D033
:10219C00514B1B69504A43F00103136110E04E4B45
:1021AC001B69184605F044F9212000F0F3F92120B1
:1021BC0000F0F0F9212000F053FA212000F050FA41
:1021CC00454B5B69444A23F002035361464B1B6841
:1021DC009AB2464BA3F85420454B0293434B0193C0
:1021EC003D4B5B693C4A43F00103536100238DF87E
:1021FC000F3053E0019B1B880093019B023301932A
:10220C00019B1B881B04009A13430093019B023310
:10221C000193029B009A1A60029B04330293019B68
:10222C001B880093019B02330193019B1B881B04A9
:10223C00009A13430093019B02330193029B009A73
:10224C001A60029B0433029300BF234B1B6903F4F7
:10225C008033002BF9D1204B1B6903F00103002BB9
:10226C0006D01D4B1B691C4A43F00103136110E09F
:10227C00194B1B69184605F0DBF8212000F08AF990
:10228C00212000F087F9212000F0EAF9212000F04C
:10229C00E7F99DF80F3001338DF80F309DF80F30B2
:1022AC00152BA7D90C4B5B690B4A23F00103536127
:1022BC00094B5B69084A43F0004353610A20FEF75F
:1022CC003BFD0C4B1B6843F07F430A4A136000BF75
:1022DC0005B05DF804FB00BF0020024023016745F8
:1022EC00AB89EFCD7A000001904100206C400020BA
:0822FC00007800089C4100205D
:1023040000B583B09D4B1B6E9C4A43F48043136617
:102314004FF090431B684FF0904223F480131360F6
:10232400974B1B68964A23F4805313604FF09043F5
:102334001B684FF0904243F400131360904B1B68EA
:102344008F4A43F4005313604FF090435B6A4FF09D
:10235400904223F4706353624FF090435B6A4FF0F2
:10236400904243F4E0635362854B1B6A844A23F032
:1023740070631362824B1B6A814A43F0E063136209
:10238400804B814A1A60814B7F4A1A60804B1B68DC
:10239400002B70D17F4B1B88602B46D0602B61DCF7
:1023A400262B3FDC0B2B5DDB0B3B1B2B5AD801A2EE
:1023B40052F823F061240008692400086924000805
:1023C40069240008692400086924000869240008B5
:1023D40069240008392400086924000869240008D5
:1023E4006924000869240008692400086924000895
:1023F4006924000869240008692400086924000885
:10240400692400084324000869240008692400089A
:102414006924000869240008692400086924000864
:102424004D240008392B14D01CE04FF41C63ADF884
:1024340006301BE04FF49C63ADF8063016E04FF411
:102444004073ADF8063011E04FF41C73ADF806305C
:102454000CE04FF4D073ADF8063007E0D023ADF8AC
:10246400063003E0D023ADF8063000BF4A4ABDF879
:102474000630D36071E0474B5B88602B47D0602BFC
:1024840062DC262B40DC0B2B5EDB0B3B1B2B5BD86F
:1024940001A252F823F000BF452500084D2500088D
:1024A4004D2500084D2500084D2500084D25000840
:1024B4004D2500084D2500081D2500084D25000860
:1024C4004D2500084D2500084D2500084D25000820
:1024D4004D2500084D2500084D2500084D25000810
:1024E4004D2500084D250008272500084D25000826
:1024F4004D2500084D2500084D2500084D250008F0
:102504004D25000831250008392B14D01CE04FF468
:102514001C63ADF806301CE04FF49C63ADF8063044
:1025240017E04FF44073ADF8063012E04FF41C731B
:10253400ADF806300DE04FF4D073ADF8063008E086
:10254400D023ADF8063004E04FF44073ADF8063004
:1025540000BF114ABDF80630D3600F4B4FF4003270
:102564005A600D4B00229A600B4B2D221A602520D5
:10257400FDF708FE00BF03B05DF804FB0010024045
:102584000004004870410020143000206C410020F9
:0C259400444100206C4000200038014051
:1025A00082B003468DF8073000BF074BDB6903F0AC
:1025B0008003002BF9D0044B9DF8072092B21A85B6
:0C25C00000BF02B0704700BF00380140AF
:1025CC0000B583B0214B9B6D204A43F400339365D7
:1025DC004FF090431B684FF0904223F05003136070
:1025EC004FF090431B684FF0904243F0A0031360F0
:1025FC004FF090431B6A4FF0904223F47F431362D9
:10260C004FF090431B6A4FF0904243F4EE43136239
:10261C000F4B104A1A60104B0E4A1A60D023ADF8BB
:10262C0006300E4ABDF80630D3600C4B00225A60BF
:10263C000A4B00229A60094B2D221A602620FDF7C6
:10264C009DFD00BF03B05DF804FB00BF001002400D
:10265C006841002014200020644100200044004008
:10266C0082B003468DF8073000BF074BDB6903F0DF
:10267C008003002BF9D0044B9DF8072092B21A85E9
:0C268C0000BF02B0704700BF00440040D7
:1026980000B583B003468DF80730114B1B68772BC4
:1026A80003D00F4B1B68002B09D19DF80730184643
:1026B800FFF772FF9DF807301846FFF7D3FF084B66
:1026C8001B68FF2B03D0064B1B68002B04D19DF819
:1026D8000730184601F08CFD00BF03B05DF804FB1D
:0426E800804100200D
:1026EC0000B585B003468DF807309DF807303033C0
:1026FC008DF80F309DF80F30392B04D99DF80F3021
:10270C0007338DF80F30114B1B68772B03D00F4B11
:10271C001B68002B09D19DF80F301846FFF73AFFC4
:10272C009DF80F301846FFF79BFF084B1B68FF2BDB
:10273C0003D0064B1B68002B04D19DF80F301846B4
:10274C0001F054FD00BF05B05DF804FB8041002092
:10275C0000B585B00346ADF80630BDF80630092B40
:10276C0065D9BDF80630632B44D9BDF80630B3F5F6
:10277C007A7F1DD3BDF80630354AA2FB03239B0993
:10278C009BB20393039B9BB21A465201D21A92003E
:10279C001344DB009BB2BDF80620D31AADF806300B
:1027AC00039BDBB23033DBB21846FFF76FFF00E060
:1027BC0000BFBDF80630274AA2FB03235B099BB27E
:1027CC000393039B9BB21A46920013441A46910042
:1027DC001A460B4613449B009BB2BDF80620D31A35
:1027EC00ADF80630039BDBB23033DBB21846FFF793
:1027FC004DFF00E000BFBDF80630174AA2FB0323D3
:10280C00DB089BB20393039B9BB21A4692001344C2
:10281C005B009BB2BDF80620D31AADF80630039BC3
:10282C00DBB23033DBB21846FFF730FF00E000BFFD
:10283C00BDF80630DBB23033DBB21846FFF726FFAB
:10284C002020FFF723FF00BF05B05DF804FB00BF9D
:0C285C00D34D62101F85EB51CDCCCCCCCD
:1028680000B583B0154B1B68002B01D1FEF77AFA2F
:10287800134B1A68134B1B689A421AD0104B1B68EB
:102888005A1C0F490A601B7843F4004301930C4B10
:102898001A680D4B1B689A4202D1094B0B4A1A6001
:1028A8000B4B4FF480329A610A4BC8221A60019B85
:1028B80000E00023184603B05DF804FB84410020C3
:1028C8006C410020704100200C00002014300020D2
:0828D8000008004898410020AF
:1028E00000B583B0154B1B68002B01D1FEF73EFAF3
:1028F000134B1A68134B1B689A421AD0104B1B6873
:102900005A1C0F490A601B7843F4404301930C4B57
:102910001A680D4B1B689A4202D1094B0B4A1A6088
:102920000B4B4FF480329A610A4BC8221A60019B0C
:1029300000E00023184603B05DF804FB844100204A
:10294000644100206841002008000020142000207D
:08295000000800489841002036
:1029580000B583B0164B1B68FF2B03D0144B1B68C4
:10296800002B07D101F09EFA03460193002B01D0FA
:10297800019B18E00E4B1B68772B03D00C4B1B6890
:10298800002B0FD1FFF76CFF03460193002B01D0FA
:10299800019B08E0FFF7A0FF03460193002B01D03D
:1029A800019B00E00023184603B05DF804FB00BF5C
:0429B800804100203A
:1029BC00364B1B68002B0AD0344B1B68B3F5004F09
:1029CC0005D2324B1B68013B304A136002E02F4B9F
:1029DC0000221A602E4B1B68002B04D02C4B1B685A
:1029EC00013B2B4A13602B4B1B68002B04D0294B4B
:1029FC001B68013B274A1360274B1B68002B04D034
:102A0C00254B1B68013B244A1360244B1B68002B8D
:102A1C0004D0224B1B68013B204A1360204B1B68DF
:102A2C00002B05D01E4B1B68013B1D4A136010E0A8
:102A3C001C4B1B68032B09D11A4BFF221A601A4B33
:102A4C00FF221A60194B77221A6002E0154B002204
:102A5C001A60174B1B68002B05D0154B1B68013BEC
:102A6C00134A136010E0104B1B68032B09D10D4B5C
:102A7C00FF221A600C4BFF221A600C4BFF221A60CB
:102A8C0002E0094B00221A6000BF7047844100200D
:102A9C009841002088410020A84100207841002066
:102AAC00944100207C4100204C41002080410020BA
:042ABC006041002055
:102AC0000D4BDB6903F02003002B12D00A4B9B8CCB
:102AD00098B20A4B1B685A1C08490A60C2B21A70A5
:102AE000064B1A68064B1B689A4202D1034B054AF3
:102AF0001A6000BF704700BF0038014070410020DD
:082B00000C000020143000203D
:102B08000D4BDB6903F02003002B12D00A4B9B8C82
:102B180098B20A4B1B685A1C08490A60C2B21A705C
:102B2800064B1A68064B1B689A4202D1034B054AAA
:102B38001A6000BF704700BF004400406841002091
:082B4800080000201420002009
:102B500082B003468DF807309DF90730002B0CDB5F
:102B60009DF8073003F01F0205499DF907305B0906
:102B7000012000FA02F241F8232000BF02B07047A2
:042B800000E100E090
:102B840082B003468DF807309DF90730002B13DB24
:102B94009DF8073003F01F0209499DF907305B09CE
:102BA400012000FA02F2203341F82320BFF34F8FB3
:102BB40000BFBFF36F8F00BF00BF02B0704700BFFC
:042BC40000E100E04C
:102BC80008B54FF090435B6A4FF0904223F47F239F
:102BD80053624FF090431B684FF0904223F070739C
:102BE80013604320FFF7CAFF084BDB6A074A43F428
:102BF8008053D362054BDB6C044A23F48053D364BF
:102C0800034B00221A6000BF08BD00BF001002403D
:042C1800484100200F
:102C1C0008B5734BDB6A724A43F48053D362704B32
:102C2C00DB6A6F4A23F48053D3626D4BDB6C6C4AC6
:102C3C0023F48053D3646B4B5B686A4A43F4806320
:102C4C0053604FF090435B6A4FF0904223F47F2324
:102C5C0053624FF090435B6A4FF0904243F42A2347
:102C6C0053624FF090431B684FF0904223F0A073D7
:102C7C0013604FF090431B684FF0904243F0207369
:102C8C0013604FF090439B684FF0904223F07073A9
:102C9C0093604FF090439B684FF0904243F0A073C9
:102CAC0093604FF09043DB684FF0904223F07073C9
:102CBC00D3604B4BDB6C4A4A43F48053D3644FF0E4
:102CCC00A0439B684FF0A04223F001039360464B56
:102CDC0003221A6000BF4FF0A0431B69002BFADAE5
:102CEC004FF0A0431B694FF0A04243F00103136166
:102CFC000120FEF721F800BF4FF0A0431A693B4BAF
:102D0C001340B3F1004FF7D10120FEF715F8364B05
:102D1C005B68354A23F0020353600220FEF70CF87F
:102D2C004FF0A0431B684FF0A04243F040031360E8
:102D3C004FF0A0431B684FF0A04243F08003136098
:102D4C004FF0A0434FF480329A633220FDF7F4FF2A
:102D5C004FF0A043DB684FF0A04243F0804343F4B4
:102D6C001153D3603220FDF7E7FF4FF0A0434FF033
:102D7C00FF325A614FF0A0431D4A9A611D4B00224D
:102D8C001A60194B00221A61174B00225A61164B1C
:102D9C000022DA6100F030F800BF4FF0A0435B690D
:102DAC0023F40053002BF8D000BF4FF0A0435B6915
:102DBC0023F48053002BF8D04FF0A0435B694FF005
:102DCC00A04243F440535361074B5B68064A43F4FB
:102DDC00807353604320FFF7B5FE00BF08BD00BFF2
:102DEC0000100240007000400008005001000080FC
:082DFC00083C0080000E0050AD
:102E04007C4B00221A607C4B03221A604FF0A043D3
:102E140080225A62794B7A4A1A607A4B7A4A1A604B
:102E24007A4B00221A607A4B1B68002B02D1794B33
:102E3400794A1A604FF0A0431B694FF0A04243F057
:102E44003003136100BF4FF0A0431B6903F030034C
:102E5400002BF8D1714B00221A60714B1B68704A29
:102E640043F05B0313606F4B00221A606E4B4FF00C
:102E740000421A606D4B1B686C4A43F05B0313609D
:102E84006B4B6C4A1A606C4B6C4A1A606C4B1B6837
:102E94006B4A43F05B0313606A4B00221A606A4B6F
:102EA4004FF480021A60694B1B68684A43F05B0365
:102EB4001360674B00221A60664B4FF400021A60DD
:102EC400654B1B68644A43F05B031360634B002249
:102ED4001A60634B634A1A60634B1B68624A43F08F
:102EE4005B031360614B624A1A60494B1B68002BF9
:102EF40019D1604B604A1A60604B1B685F4A43F00B
:102F04005B0313605E4B00221A605E4B4FF4400279
:102F14001A605D4B1B685C4A43F05B0313605B4BB8
:102F240000221A6017E0534B00221A60534B1B68AF
:102F3400524A43F05B031360514B00221A60514B19
:102F440000221A60504B1B684F4A43F05B03136026
:102F54004E4B00221A60284B5B69274A43F0090351
:102F64005361254B1B69244A43F0190313614FF045
:102F7400A04300229A614FF0A0434FF0FF325A6100
:102F84004FF0A0439A694FF0A041414B13438B612A
:102F94004FF0A0439B684FF0A04243F0810393603D
:102FA400154B3C4ADA611A4B1B68002B05D1124BB6
:102FB400DB69114A43F00803D3610F4B00225A63C3
:102FC400354B00221A60354B00221A80344B354AA7
:102FD4001A60354B334A1A60344B354A1A60354B04
:102FE400334A1A60344B00221A70344B00221A7090
:102FF40000BF7047484100200008005028000050DE
:10300400800040000401005000014000080100500D
:10301400444100200C0100508001200000090050B0
:103024000809005010090050000B0050080B005014
:10303400100B005040000860200900504000480078
:103044002809005030090050200B0050280B005074
:10305400300B0050400900504809005050090050FE
:10306400400B005040008800480B0050500B0050AB
:1030740040000800600900501000CC0068090050AE
:1030840070090050600B0050680B0050700B00502A
:1030940018380C00030005003C410020B04100201A
:1030A4005441002014000020504100205C410020C5
:1030B4001410002058410020B6410020B8410020DF
:1030C40000B587B04FF0A0439B694FF0A04223F0B6
:1030D40010039361924B05934FF0A0431B6A039333
:1030E400039A904B13400293039B03F00F03002BAE
:1030F4003FD1029B029B8C4A93420BD1059B1B68D8
:103104000293059B1B680193884B20221A60884B0D
:1031140000221A80039B03F4F013B3F5402F28D147
:10312400059B1B680293059B1B680193029BDAB203
:10313400804B1A70029B1B0ADAB27F4B1A70029BF7
:103144001B0C9AB27D4B1A807C4B1B881B0A9BB2CA
:10315400DAB27B4B1A70794B1B88DAB2794B1A704E
:10316400019B9AB2784B1A80019B1B0C9AB2774B45
:103174001A80039A764B1340764A934240F0C480F7
:10318400039B1B09DAB2744B1A7086E0059B1B681B
:103194000293724B1B68012B04D1029B184600F06A
:1031A400F7FE7AE0029B8DF813306D4B1B685A1CB6
:1031B4006B490A609DF813201A70694B1A68694BB1
:1031C4001B689A4202D1664B674A1A60624B1B78AD
:1031D400013BDAB2604B1A705F4B1B78002B6CD04A
:1031E400029B1B0A8DF813305D4B1B685A1C5C490B
:1031F4000A609DF813201A70594B1A68594B1B68C2
:103204009A4202D1564B584A1A60534B1B78013BE1
:10321400DAB2514B1A70504B1B78002B4FD0029BE3
:103224001B0C8DF813304E4B1B685A1C4C490A601A
:103234009DF813201A704A4B1A684A4B1B689A422D
:1032440002D1474B484A1A60434B1B78013BDAB220
:10325400414B1A70404B1B78002B32D0029B1B0E43
:103264008DF813303E4B1B685A1C3D490A609DF88B
:1032740013201A703A4B1A683A4B1B689A4202D1CF
:10328400374B394A1A60344B1B78013BDAB2324B64
:103294001A70314B1B78002B15D02F4B1B78194615
:1032A4002E4B1A6813465B00134499420CD92A4BDF
:1032B4001B78402B7FF66AAF06E000BF04E000BF36
:1032C40002E000BF00E000BF284B1A68244B1B68D3
:1032D4009A4208D9224B1B6803F6FE72234B1B68E3
:1032E400D31A009305E01E4B1A68204B1B68D31AAF
:1032F40000931F4B00221A60009B40F6B872934261
:1033040002D91B4BFF221A604FF0A0439B694FF078
:10331400A04243F01003936100BF07B05DF804FBC3
:1033240000100050FF7F1E00700004003C4100208C
:10333400B0410020BA410020BB4100201E410020C2
:10334400C3410020C4410020B4410020B241002008
:103354000F001E0002000400B94100204441002077
:103364005C4100200400002014100020584100207B
:0433740040410020B4
:1033780000B583B0784B9B69DAB2774BDB69DBB277
:103388001340DBB28DF807309DF80730DBB203F04D
:103398000103002B00F086806F4B1A696E4B5B6B44
:1033A800DB0103F08003134300936C4B1A68009B06
:1033B80013400093009B03F08003002B13D0664B4F
:1033C8005B6B654A23F001035363654B1B68012B54
:1033D80007D0634B1B68062B03D0614B1B68A12BDE
:1033E80001D100F04DFC009B03F00103002B49D0F4
:1033F8005A4B01221A605B4B1B88002B30D1584B6B
:103408001B68052B0BD0564B1B68092B07D0544B58
:103418001B68222B03D0524B1B68202B10D1524B18
:103428001B68002B0CD1514B514A1A60514B524A20
:103438001A60524B1B68002B02D1514B514A1A603B
:10344800454B5B6B444A23F0010353634E4B4F4A91
:103458001A604F4B1B684E4A43F00443136011E057
:10346800404B1B8843F400224A4B1A604A4B1B68A6
:10347800494A43F004431360374B5B6B364A43F0C9
:1034880001035363009B03F01003002B02D0334B5E
:1034980010221A60009B03F00803002B02D02F4B68
:1034A80008221A609DF80730DBB203F00203002BF4
:1034B80000F0AD80284B1A69274B5B6B9B0103F02A
:1034C800800313430093354B1A68009B1340009305
:1034D800009B03F08003002B07D01F4B5B6B1E4A39
:1034E80023F00203536300F03BFC009B03F001034D
:1034F800002B04D1009B03F01003002B7FD0009B0E
:1035080003F00103002B02D0244B01221A60244B44
:103518001A68244B1B689A420CD1144B1B68134A37
:1035280043F0044313600C4B5B6B0B4A23F002031C
:1035380053635CE01A4B1A681A4B1B689A4235D9D8
:10354800184B1B6803F6FE72154B1B68D31A9AB208
:10355800154B1A8032E000BF0008005008090050DF
:103568003C410020B0410020484100202009005083
:1035780040804884400B00504080888444410020AB
:10358800600900501080CC84100B00504000086087
:10359800000B005010090050000900502809005085
:1035A800504100205441002032410020484B1A6805
:1035B800484B1B68D31A9AB2474B1A80464B1B8854
:1035C800402B02D9444B40221A80434B1B8843F4BA
:1035D8000022424B1A60424B1B68414A43F00443A5
:1035E8001360404B5B6B3F4A43F002035363009BFD
:1035F80003F01003002B02D03B4B10221A60009BF3
:1036080003F00803002B02D0374B08221A609DF8FC
:103618000730DBB203F00803002B54D0314B1A6992
:10362800304B5B6B1B0103F08003134300932F4B5C
:103638001A68009B13400093009B03F08003002B43
:1036480009D02B4B4FF400221A602A4B1B68294AD9
:1036580043F004431360009B03F00103002B12D0D6
:10366800234B4FF400221A60224B1B68214A43F077
:10367800044313601D4B01221A601A4B5B6B194AF5
:1036880023F008035363009B03F01003002B12D0B0
:10369800174B4FF400221A60164B1B68154A43F06B
:1036A800044313600F4B5B6B0E4A23F0080353630C
:1036B8000E4B10221A60009B03F00803002B02D067
:1036C8000A4B08221A6000BF03B05DF804FB00BF74
:1036D8005441002050410020324100203009005060
:1036E80020090050000800502809005068090050BF
:0836F800700900506009005048
:1037000000B583B0774B9A69764BDB6913401B0C8D
:10371000DBB28DF807309DF80730DBB203F0010310
:10372000002B00F0AB80704B1B68DAB26D4B5B690D
:10373000DBB21340DBB28DF806309DF80630DBB209
:1037400003F00103002B2AD0674B01221A60674B5C
:10375000674A1A60674B1B68664A43F0044313606C
:10376000654B1B78802B0CD1644B1B78002B08D148
:103770009DF80630DBB243F00803DBB28DF806306B
:103780000DE05F4B1B68202B09D15E4B4FF40022EC
:103790001A605D4B1B685C4A43F0044313609DF85C
:1037A0000630DBB203F00803002B00F0978000F036
:1037B000BBF8534B1B68052B1BD14A4B1B68534A64
:1037C000127812011146474A0B4313604D4B4FF4D8
:1037D00000221A604C4B1B684B4A43F004431360B1
:1037E000414B08221A603F4B5B6B3E4A43F001039A
:1037F0005363434B1B68092B03D0414B1B68222B9F
:1038000012D1404B4FF400221A603F4B1B683E4AD6
:1038100043F004431360344B08221A60314B5B6B56
:10382000304A43F001035363354B1B68012B07D02B
:10383000334B1B68062B03D0314B1B68A12B4DD19A
:10384000334B1B88402B03D92E4B324A1A6005E0BC
:103850002F4B1B8843F400222A4B1A602A4B1B680B
:10386000294A43F0044313601F4B08221A601D4B82
:103870005B6B1C4A43F0010353632FE09DF8073054
:10388000DBB203F00403002B29D0234B1B68DAB210
:10389000144B5B69DBB21340DBB28DF806309DF848
:1038A0000630DBB203F00103002B18D01A4B0122C3
:1038B0001A601A4B174A1A60194B1B68002B06D165
:1038C000184B1B68174A43F00443136007E0154B7D
:1038D0001B68144A43F00043136000E000BF03B0CC
:1038E0005DF804FB00080050080B0050100B00505E
:1038F00040000860000B0050BA410020BB4100208E
:103900003C4100201009005000090050C541002032
:10391000B041002040000800480B0050500B005000
:0839200040410020400B005063
:1039280000B583B0904B00221A60904B1B78212B76
:1039380024D18F4B1B78202B12D18E4B1B688D4ABC
:1039480043F0080313608C4B8C4A1A608C4B1B683D
:103958008B4A43F004431360834B20221A606EE1C4
:10396800834B1B78222B06D17F4B22221A60854B72
:1039780000221A8063E100F0E9F960E17B4B1B78D3
:10398800A12B17D17A4B1B78212B13D1764BA1226F
:103998001A607C4B07221A807B4B1A88794B1B884C
:1039A8009A4203D2784B1A88764B1A80774B784A1A
:1039B8001A6044E16D4B1B7803F06103002B06D0BD
:1039C8006A4B1B7803F06103012B40F03681684B8A
:1039D8001B78092B00F22A8101A252F823F000BFBC
:1039E800113A0008353C0008353C0008353C000811
:1039F800353C0008393A0008573A0008353C0008B9
:103A0800353C0008073C0008574B01221A605D4B03
:103A180002221A805C4B1A885A4B1B889A4203D29E
:103A2800594B1A88574B1A80584B5A4A1A6003E167
:103A3800594B1B88DBB203F07F03DAB2574B1A707D
:103A4800494B05221A604F4B00221A80F4E0464B7E
:103A580006221A60524B1B78012B65D1494B122262
:103A68001A80494B1A88474B1B889A4203D2464B07
:103A78001A88444B1A804B4B1B68012B03D1434BCC
:103A8800494A1A6002E0414B484A1A60484B009381
:103A98000023ADF806300EE03C4B1A68531C3B4936
:103AA8000B60009B591C009112781A70BDF8063003
:103AB8000133ADF80630BDF80630112BECD93D4B7B
:103AC8001A893C4B5B8913439AB23A4B9B8913433F
:103AD8009AB2384BDB891343ADF80630BDF806308F
:103AE800002B1DD0334B5B89DAB2314B1A72314B44
:103AF8001B89DAB22E4B5A722E4BDB89DAB22C4B69
:103B08009A722C4B9B89DAB2294BDA72254B1B68C7
:103B1800012B05D1264B9B7A0233DAB2244B9A72D9
:103B28001A4B234A1A6084E01D4B1B78022B47D19D
:103B38001C4B1B68012B06D1124B65221A80134BB4
:103B48001D4A1A6005E00F4B43221A800F4B1B4A8F
:103B58001A600D4B1A880B4B1B889A4269D20A4B84
:103B68001A88084B1A8064E03C410020BA410020C2
:103B7800BB410020080B0050100B005040000860AB
:103B8800000B0050B0410020B24100203841002015
:103B980054730008D06D00081E410020C541002064
:103BA800C3410020444100204C6E00087C6D000891
:103BB8000C4100206C400020F470000810730008CD
:103BC800204B1B78032B17D11F4B1B78012B10D1CF
:103BD8001E4B18221A801E4B1A881C4B1B889A42AF
:103BE80003D21B4B1A88194B1A801A4B1A4A1A60AF
:103BF8001FE000F0ABF822E000F0A8F819E0174B3E
:103C080009221A60114B00221A80154BFF221A60F4
:103C1800144B154A1A60154B154A1A60154B1B6848
:103C2800002B08D1144B154A1A6004E000F08EF8F6
:103C380002E000BF03E000BF01E000F087F803B036
:103C48005DF804FBC3410020C4410020B0410020BE
:103C5800B241002038410020D06600083C410020D5
:103C6800484100202009005040804884400B005003
:103C78004080888444410020600900501080CC8432
:103C880084B02F4B1B88402B11D92E4B1B680393F4
:103C98002C4B1B6840332B4A136040238DF80330AC
:103CA800274B1B88403B9AB2254B1A800AE0254BCC
:103CB8001B680393224B1B88DBB28DF80330204B23
:103CC80000221A809DF80330DBB20333002B00DAA0
:103CD80003339B10DBB28DF802301B4B0293002399
:103CE8008DF801301FE0039B03331B781B061A462F
:103CF800039B02331B781B041343039A0132127887
:103D080012021343039A127813430193019A029BF8
:103D18001A60039B043303939DF80130DBB201332F
:103D2800DBB28DF801309DF80130DAB29DF802302F
:103D3800DBB29A42D7D300BF00BF04B0704700BFC0
:0C3D4800B0410020384100200010005065
:103D5400034B1B68024A43F40013136000BF70470F
:043D6400000B005000
:103D680086B04A4B05934A4B1B6804937FE0494B46
:103D78001B681B780393474B1B680133454A136044
:103D8800444B1A68444B1B689A4202D1414B434A40
:103D98001A60434B1B88013B9AB2414B1A8000239F
:103DA800029300230193002300933D4B1B88002BB3
:103DB80017D0384B1B681B780293364B1B680133AE
:103DC800344A1360334B1A68334B1B689A4202D14A
:103DD800304B324A1A60324B1B88013B9AB2304B47
:103DE8001A802F4B1B88002B17D02A4B1B681B7877
:103DF8000193284B1B680133264A1360254B1A6828
:103E0800254B1B689A4202D1224B244A1A60244B44
:103E18001B88013B9AB2224B1A80214B1B88002B2E
:103E280017D01C4B1B681B7800931A4B1B68013377
:103E3800184A1360174B1A68174B1B689A4202D12D
:103E4800144B164A1A60164B1B88013B9AB2144B46
:103E58001A80009B1A06019B1B041A43029B1B0233
:103E68001A43039B13430493049A059B1A600C4B53
:103E78001B88002B7FF47BAF00BF054B1B68402BD2
:103E8800FBD100BF00BF06B0704700BF0020005044
:103E98003809005050410020000000201400002084
:043EA8003241002083
:103EAC0000B583B0304B1B68002B01D1FCF758FFD9
:103EBC002E4B1B68002B01D1002350E02C4B1A68B1
:103ECC002C4B1B689A4249D0FCF728FF284B1B68E7
:103EDC005A1C27490A601B781BB26FEA43436FEAEE
:103EEC0053431BB29BB2ADF80630214B1A68224BE0
:103EFC001B689A4202D11E4B204A1A601C4B1A684E
:103F0C001C4B1B689A420CD91A4B1B681A46184B4F
:103F1C001B68D31A9BB203F6FE739BB2ADF8043048
:103F2C0008E0144B1B681A46114B1B68D31A9BB242
:103F3C00ADF80430BDF804309BB240F6B772934232
:103F4C0008D80F4B00221A600E4B1B680D4A43F029
:103F5C0004431360BDF806309BB200E00023184602
:103F6C0003B05DF804FB00BF8441002048410020F1
:103F7C00584100205C410020040000201410002057
:083F8C0040410020400B0050F1
:103F940000B585B00190019B8DF80F30904B1B78D4
:103FA400013BDAB28E4B1A708D4B1B78002B01D17A
:103FB400002311E1019B1B0A8DF80E30884B1B78FE
:103FC400013BDAB2864B1A70854B1B78002B01D16A
:103FD400002301E1019B1B0C8DF80D30804B1B78F5
:103FE400013BDAB27E4B1A707D4B1B78002B01D15A
:103FF4000023F1E0019B1B0E8DF80C30784B1B78ED
:10400400013BDAB2764B1A709DF80F300F2B01D9B1
:104014000023E1E09DF80F30012B01D80023DBE001
:10402400FCF780FE9DF80F30052B03D09DF80F3070
:104034000F2B15D16B4B00221A706B4B1B685A1C4B
:1040440069490A609DF80E201A70674B1A68674B1D
:104054001B689A4202D1644B654A1A600123BBE093
:104064009DF80F300C2B03D09DF80F300D2B2DD164
:104074005C4B1B789DF80E209A4214D05A4B1B6857
:104084005A1C59490A609DF80E201A70564B1A683A
:10409400564B1B689A4202D1534B554A1A60514AF7
:1040A4009DF80E301370504B1B685A1C4E490A6021
:1040B4009DF80D201A704C4B1A684C4B1B689A42A1
:1040C40002D1494B4A4A1A60012385E09DF80F301A
:1040D400022B03D09DF80F30062B26D1414B002232
:1040E4001A70414B1B685A1C3F490A609DF80E2008
:1040F4001A703D4B1A683D4B1B689A4202D13A4BE9
:104104003B4A1A60384B1B685A1C37490A609DF8B1
:104114000D201A70344B1A68344B1B689A4202D132
:10412400314B334A1A60012356E09DF80F30072BB8
:1041340014D82C4B00221A702B4B1B685A1C2A498A
:104144000A609DF80E201A70274B1A68274B1B68CB
:104154009A421ED1244B264A1A601AE0214B1B783E
:104164009DF80E209A4214D01F4B1B685A1C1E49FE
:104174000A609DF80E201A701B4B1A681B4B1B68B3
:104184009A4202D1184B1A4A1A60164A9DF80E3008
:104194001370154B1B685A1C13490A609DF80D20B7
:1041A4001A70114B1A68114B1B689A4202D10E4BBC
:1041B4000F4A1A600C4B1B685A1C0B490A609DF885
:1041C4000C201A70084B1A68084B1B689A4202D1DB
:1041D400054B074A1A600123184605B05DF804FB35
:1041E400B9410020B84100205C41002004000020B7
:0441F4001410002083
:1041F80082B003468DF807300C4B1B68002B11D09A
:104208000B4B1B685A1C0A490A609DF807201A7054
:10421800074B1A68074B1B689A4204D1044B064A9D
:104228001A6000E000BF02B0704700BF484100209C
:0C42380054410020000000201400002071
:1042440084B003468DF80730A74B1B780133DAB2EC
:10425400A54B1A709DF90730002B80F2EF809DF872
:104264000730F72B02D0A04B01221A709DF80730BB
:10427400F02B0FD19D4BF0221A709D4BFF221A7028
:104284009C4B00221A709C4B00221A709B4B0022FC
:104294001A700BE29DF80730F72B40F08780924BA1
:1042A4001B78012B35D1964B05221A708F4BF722C0
:1042B4001A70944B00221A70934B00221A708C4B84
:1042C40000221A708B4B00221A708B4B00221A703A
:1042D4008A4B1B78002B0CD0844BF7221A70894B25
:1042E40000221A70884B00221A70844B00221A7024
:1042F40084E17F4B00221A707B4B00221A707D4BA5
:1043040000221A707C4B00221A707C4B00221A7017
:10431400CCE1754B1B78022B21D1794B06221A7004
:10432400724B1B78F02B03D0764B1A786F4B1A70B4
:10433400744B1A786D4B1A70724BF7221A70724BC9
:1043440000221A706A4B00221A706A4B00221A70FB
:10435400694B00221A70694B00221A704EE1684BB7
:1043640007221A70614B1B78F02B07D1634B1B7823
:10437400002B03D1644BF7221A700AE0614B1A78C0
:104384005A4B1A70604B1A785E4B1A705E4BF722C8
:104394001A70574B00221A70564B00221A70564B53
:1043A40000221A70554B00221A7027E14F4A9DF8DB
:1043B400073013704D4B1B78F32B0CD84C4BFF225A
:1043C4001A704C4B00221A704B4B00221A704B4B44
:1043D40000221A706AE1454B1B78F42B0BD0434B37
:1043E4001B78F52B07D0414B1B78F92B03D03F4B9F
:1043F4001B78FD2B0CD13E4B00221A703D4B002242
:104404001A703D4B00221A703C4B00221A704DE189
:104414003B4B05221A703B4B00221A703A4B002288
:104424001A70334B00221A70324B00221A70324B2E
:1044340000221A70314B00221A70DFE02B4B1B78DC
:1044440023F00F038DF80B30294B1B78002B0CD174
:10445400254B00221A70274B00221A70264B00228B
:104464001A70264B00221A7020E1224B1B78002B75
:1044740050D1244A9DF807301370234B00221A7040
:104484001A4B1B78F12B03D0184B1B78F32B0FD14D
:104494001B4B02221A70164B00221A70154B002275
:1044A4001A70154B00221A70144B00221A70A5E0E2
:1044B4009DF80B30C02B03D09DF80B30D02B25D1A9
:1044C4009DF80B301B09DAB20D4B1A70084BFF2212
:1044D4001A70084B00221A70074B00221A70074BFF
:1044E40000221A708AE000BFB6410020BE410020BD
:1044F400BD410020C2410020C1410020B74100203D
:10450400BC410020C0410020BF410020684BFF2275
:104514001A70CBE0674B1B78002B0CD1664B002242
:104524001A70634B00221A70644B00221A70644B99
:1045340000221A70BAE0614B1B78002B43D1614A08
:104544009DF8073013705E4B1B78002B03D05B4B38
:10455400FF221A70AAE05C4B1B78F22B0FD15B4B45
:1045640003221A70534B00221A70514B00221A7006
:10457400524B00221A70524B00221A703EE0524BEA
:104584001B78F02B0FD1514B04221A704C4BFF2295
:104594001A70484BFF221A70454B00221A70474B81
:1045A40000221A702AE09DF80B301B09DAB2474B3F
:1045B4001A70404BFF221A703D4B00221A703F4B79
:1045C40000221A701AE0424B1A783F4B1A703D4B86
:1045D4001A783F4B1A703B4A9DF8073013703B4BD7
:1045E40004221A70364BFF221A70324BFF221A70C3
:1045F4002F4B00221A70314B00221A70354B1B6866
:10460400002B52D0344B1B680393039B5A1C039218
:104614002E4A12781A70314B1B68039A9A4201D1C0
:104624002F4B0393039B5A1C0392274A12781A7048
:104634002A4B1B68039A9A4201D1294B0393039B8B
:104644005A1C0392224A12781A70244B1B68039A4C
:104654009A4201D1224B0393039B5A1C0392194A99
:1046640012781A701D4B1B68039A9A4201D11C4B95
:104674000393194A039B13600F4B00221A700C4BCF
:1046840000221A700D4B00221A70104B1B78072B56
:1046940003D80E4B1B78042B03D10B4B1B78F02B48
:1046A40004D9044B00221A7000E000BF04B0704724
:1046B400C2410020BD410020B6410020C14100207C
:1046C400B7410020BF410020BE410020BC41002072
:1046D400C041002048410020544100200000002037
:0446E400140000209E
:1046E80030B5B9B0D64B26AC1D460FCD0FC40FCD93
:1046F8000FC40FCD0FC495E80F0084E80F00D14B0D
:104708001EAC1D460FCD0FC495E80F0007C42380CB
:10471800CD4B16AC1D460FCD0FC495E80F0007C44E
:104728002370CA4B12AC0FCB07C42370C84B08AC1C
:104738001D460FCD0FC40FCD0FC495E8030084E8C4
:104748000300C44B04AC0FCB84E80F00C24B6C468B
:104758000FCB07C4238002341B0C237002F0C5FB67
:10476800BE4802F0D3FE3320FDF792FF2E20FDF75E
:104778008FFF3620FDF78CFFB94802F0C7FE4FF4D3
:104788007A70FCF7DBFA00238DF8DF3002F0ADFB1E
:104798004320FDF77DFF4D20FDF77AFF4420FDF70C
:1047A80077FF3E20FDF774FF00BFFEF7D1F8034600
:1047B800ADF8DC30BDF8DC30002BF6D0BDF8DC30CD
:1047C8008DF8DF309DF8DF30202BEDD09DF8DF30FD
:1047D8000A2B00D1E8E79DF8DF30602B08D99DF857
:1047E800DF307A2B04D89DF8DF30203B8DF8DF309E
:1047F8009DF8DF30302B14D99DF8DF30392B10D8D5
:104808006B46184602F082FE9DF8DF301846FDF729
:104818003FFF9DF8DF30312B0ED03A20FDF738FFEF
:104828000AE09DF8DF301846FDF732FF3A20FDF721
:104838002FFF2020FDF72CFF9DF8DF300D3B712B5B
:1048480000F27A8201A252F823F000BF394D000825
:10485800414D0008414D0008414D0008414D0008F8
:10486800414D0008414D0008414D0008414D0008E8
:10487800414D0008414D0008414D0008414D0008D8
:10488800414D0008414D0008414D0008414D0008C8
:10489800414D0008414D0008414D00081D4A0008DF
:1048A800414D0008414D0008414D0008414D0008A8
:1048B800414D0008414D0008414D0008414D000898
:1048C800414D0008414D0008414D0008414D000888
:1048D800414D0008414D0008414D0008954A000827
:1048E800414D0008EB4A0008F34A0008FB4A00085B
:1048F800034B00080B4B0008134B00081B4B000828
:10490800414D0008414D0008414D0008414D000847
:10491800414D0008234A00082B4B0008414D000870
:104928002F4A00083B4A00086D4A00082B4C000833
:10493800414D0008414D0008414A0008414D00081A
:10494800414D0008414D0008414D0008354A000816
:10495800414D0008414D0008414D0008414D0008F7
:10496800414D0008414D0008414D0008234B000807
:10497800294A0008414D0008814A0008414D0008B5
:10498800414D0008414D0008414D0008414D0008C7
:10499800414D0008414D0008414D0008414D0008B7
:1049A800414D0008414D0008414D0008414D0008A7
:1049B800414D0008414D0008414D0008414D000897
:1049C800414D0008414D0008414D0008414D000887
:1049D800414D0008414D0008414D0008414D000877
:1049E800414D0008414D0008414D0008414D000867
:1049F800414D0008414D0008414D0008414D000857
:104A0800414D0008414D0008414D0008414D000846
:104A1800AD4B000801F0CEF992E101F097F88FE173
:104A280000F0A4F98CE100F0B7FA89E100F0E8FBA6
:104A380086E100F0F3FC83E100F082FD80E100BF35
:104A480094680008D4680008F4680008146900082D
:104A5800246900084C6900085C690008486D000872
:104A6800B8660008B84B00221A60B84802F04EFD3C
:104A7800B74802F04BFD63E1B34B01221A60B3481B
:104A880002F044FDB34802F041FD59E102F0D3FBC6
:104A980003468DF8DB309DF8DB303F2B03D13F20F8
:104AA800FDF7F6FD4CE19DF8DB300D2B03D13F20DF
:104AB800FDF7EEFD44E19DF8DB30062B03D93F20DE
:104AC800FDF7E6FD3CE13A20FDF7E2FD9DF8DB301D
:104AD8000A338DF8DB309DF8DB30184600F07CFD9A
:104AE8002EE1032000F078FD2AE1042000F074FD97
:104AF80026E1052000F070FD22E1062000F06CFDA3
:104B08001EE1072000F068FD1AE1082000F064FDAE
:104B180016E1092000F060FD12E1112000F05CFDB3
:104B28000EE10D20FDF7B4FD3E20FDF7B1FD4FF479
:104B38009670FCF703F9FDF70BFF0346002B05D031
:104B48003F20FDF7A5FD2020FDF7A2FD08AB184684
:104B580002F0DCFCFDF7FCFE0346ADF8DC30BDF8E6
:104B6800DC30002BF6D0BDF8DC3048F2400293422E
:104B780013D1FDF79DF802F0EAF82020FDF788FD33
:104B88006F20FDF785FD6B20FDF782FD2020FDF7E6
:104B98007FFD714B00221A60D2E004AB184602F088
:104BA800B5FCCDE00D20FDF773FD3E20FDF770FD4F
:104BB8004FF49670FCF7C2F8FDF7CAFE0346002BC7
:104BC80005D03F20FDF764FD2020FDF761FD16AB01
:104BD800184602F09BFCFDF7BBFE0346ADF8DC303F
:104BE800BDF8DC30002BF6D0BDF8DC3048F27C0292
:104BF800934211D1FDF79EFA2020FDF749FD6F2061
:104C0800FDF746FD6B20FDF743FD2020FDF740FD35
:104C1800514B00221A6093E012AB184602F076FC62
:104C28008EE04D4B1B6823F07F43002B65D04B4B28
:104C380001221A6026AB184602F068FC02F055F90A
:104C48001EAB184602F062FC02F04FF93E20FDF759
:104C58001FFD00BFFDF77CFE0346ADF8DC30BDF854
:104C6800DC30002BF6D0BDF8DC3048F21B02934252
:104C780003D13A4B00221A6062E0BDF8DC3048F2FA
:104C88007C02934235D14FF49670FCF757F8FDF744
:104C98005FFE0346002B05D03F20FDF7F9FC2020DE
:104CA800FDF7F6FC16AB184602F030FCFDF750FE97
:104CB8000346ADF8DC30BDF8DC30002BF6D0BDF88B
:104CC800DC3048F27C0293420ED1FDF733FA202003
:104CD800FDF7DEFC6F20FDF7DBFC6B20FDF7D8FC51
:104CE8002020FDF7D5FC08E012AB184602F00EFCB8
:104CF80003E012AB184602F009FC4520FDF7C8FC9A
:104D08007820FDF7C5FC6920FDF7C2FC7420FDF78B
:104D1800BFFC02F0EAF8124B00221A60114B002285
:104D28001A60114B00221A600C4B00221A6008E02E
:104D38000D20FDF7ADFC03E03F20FDF7A9FC00BF07
:104D480024E539B030BD00BF904100203867000825
:104D5800446700084C6700089C410020A4410020DB
:0C4D6800804100207C4100204C410020D4
:104D740030B595B0834B09AC1D460FCD0FC40FCD94
:104D84000FC42B682370804B6C461D460FCD0FC497
:104D94000FCD0FC42B6823707C4B01221A607C4B0F
:104DA40000221A6002F0A3F809AB184602F0B0FB27
:104DB400002002F0D0F903468DF847309DF84730C3
:104DC400EE2B03D1714B00221A60D8E09DF84730D6
:104DD400ADF84E30002002F0BEF903468DF847309E
:104DE4009DF84730EE2B03D1684B00221A60C6E0D1
:104DF400BDF84E301B019AB29DF847309BB2134464
:104E0400ADF84E30002002F0A6F903468DF8473085
:104E14009DF84730EE2B03D15C4B00221A60AEE0C4
:104E24009DF84730ADF84C30002002F094F9034669
:104E34008DF847309DF84730EE2B03D1534B0022B9
:104E44001A609CE0BDF84C301B019AB29DF84730C3
:104E54009BB21344ADF84C30BDF84E20BDF84C3035
:104E640013439BB2002B07D14FF6FF73ADF84E30BE
:104E74004FF6FF73ADF84C3002F039F86B46184624
:104E840002F046FB002002F066F903468DF8473035
:104E94009DF84730EE2B03D13C4B00221A606EE0A4
:104EA4009DF84730ADF84A30002002F054F903462B
:104EB4008DF847309DF84730EE2B03D1334B002259
:104EC4001A605CE0BDF84A301B019AB29DF8473085
:104ED4009BB21344ADF84A30002002F03CF903467B
:104EE4008DF847309DF84730EE2B03D1274B002235
:104EF4001A6044E09DF84730ADF84830002002F0D5
:104F04002AF903468DF847309DF84730EE2B03D13C
:104F14001E4B00221A6032E0BDF848301B019AB2E1
:104F24009DF847309BB21344ADF84830BDF84A2091
:104F3400BDF8483013439BB2002B07D14FF6FF73E3
:104F4400ADF84A304FF6FF73ADF84830114ABDF85A
:104F54004E3013810F4ABDF84C3053810D4ABDF8D1
:104F64004A3093810B4ABDF84830D3810A4B1B6801
:104F740043F47F43084A1360044B00221A6015B0BF
:104F840030BD00BF6C69000890690008A44100208E
:0C4F9400A04100206C4000209C41002047
:104FA00030B58DB0944B01AC1D460FCD0FC40FCD65
:104FB0000FC495E8030020600434218002340B0CF8
:104FC00023708E4B01221A6001F093FF01AB18464B
:104FD00002F0A0FA02F033F903468DF82F309DF865
:104FE0002F303F2B03D1854B00221A6001E19DF841
:104FF0002F308DF82E309DF82F30002B0FD09DF8DC
:105000002F30042B0BD09DF82F30062B07D09DF8A6
:105010002F30072B03D09DF82F30082B06D13F20CF
:10502000FDF73AFB754B00221A60E2E002F007F947
:1050300003468DF82F309DF82F303F2B03D16F4B57
:1050400000221A60D5E09DF82E301A4692001344D3
:105050005B00DAB29DF82F3013448DF82E309DF8A6
:105060002E30392B68DC0B2BC0F2B1800B3B2E2B82
:1050700000F2AD8001A252F823F000BF9B5100085E
:10508000CF510008CF510008CF510008CF51000880
:10509000CF510008CF510008CF5100084B510008F4
:1050A000CF510008CF510008CF510008B55100087A
:1050B000CF510008CF510008CF510008CF51000850
:1050C000CF510008CF510008CF5100085F510008B0
:1050D000CF510008CF510008CF510008CF51000830
:1050E000CF510008CF51000873510008CF5100087C
:1050F000CF510008CF510008CF510008CF51000810
:10510000CF510008CF510008CF510008CF510008FF
:10511000CF510008CF510008CF510008CF510008EF
:10512000CF510008CF510008CF510008CF510008DF
:10513000CF51000887510008602B48D13020FDF77F
:10514000ABFA3020FDF7A8FA48E03220FDF7A4FAC8
:105150003020FDF7A1FA3020FDF79EFA3EE0322024
:10516000FDF79AFA3520FDF797FA3020FDF794FA0B
:1051700034E03420FDF790FA3020FDF78DFA30202E
:10518000FDF78AFA2AE03220FDF786FA3020FDF793
:1051900083FA3020FDF780FA20E03520FDF77CFA15
:1051A0003220FDF779FA3020FDF776FA3020FDF74E
:1051B00073FA13E03020FDF76FFA3420FDF76CFA34
:1051C0003020FDF769FA3020FDF766FA06E03F204F
:1051D000FDF762FA094B00221A600AE09DF82E30B2
:1051E0009AB2074B1A80074BFF221A60034B00222A
:1051F0001A600DB030BD00BFB4690008A4410020A2
:085200006C4000209C410020DD
:1052080030B58DB0804B01AC1D460FCD0FC40FCD0E
:105218000FC495E8030084E803007C4B01221A6060
:1052280001F063FE01AB184602F070F902F003F8D2
:1052380003468DF82F309DF82F303F2B03D1734B49
:1052480000221A60DDE09DF82F308DF82E309DF891
:105258002F30002B13D09DF82F30022B0FD09DF844
:105268002F30042B0BD09DF82F30062B07D09DF83C
:105278002F30072B03D09DF82F30082B06D13F2065
:10528800FDF706FA614B00221A60BAE001F0D3FF7D
:1052980003468DF82F309DF82F303F2B03D15B4B01
:1052A80000221A60ADE09DF82E301A469200134491
:1052B8005B00DAB29DF82F3013448DF82E309DF83C
:1052C8002E30602B47D0602B00F38180262B3FDCEB
:1052D8000B2B7CDB0B3B1B2B79D801A252F823F05C
:1052E800BD530008D7530008D7530008D753000808
:1052F800D7530008D7530008D7530008D7530008DE
:105308006D530008D7530008D7530008D753000837
:10531800D7530008D7530008D7530008D7530008BD
:10532800D7530008D7530008D7530008D7530008AD
:1053380081530008D7530008D7530008D7530008F3
:10534800D7530008D7530008D753000895530008CF
:10535800392B25D03BE03020FDF79AF93020FDF7B6
:1053680097F93BE03220FDF793F93020FDF790F9EB
:105378003020FDF78DF931E03220FDF789F935202D
:10538800FDF786F93020FDF783F927E03420FDF793
:105398007FF93020FDF77CF93020FDF779F91DE021
:1053A8003220FDF775F93020FDF772F93020FDF74E
:1053B8006FF913E03520FDF76BF93220FDF768F936
:1053C8003020FDF765F93020FDF762F906E03F204F
:1053D800FDF75EF90D4B00221A6012E09DF82E30A1
:1053E8009AB20B4B5A809DF82E309AB2094B5A80CC
:1053F800094B1B6843F47F03074A1360034B0022E1
:105408001A600DB030BD00BFDC690008A44100205F
:0C5418006C400020144000209C4100204B
:1054240030B589B0424B6C461D460FCD0FC495E88C
:105434000F0007C423803F4B01221A6001F057FD7F
:105444006B46184602F064F801F0F7FE03468DF847
:105454001E309DF81E303F2B03D1364B00221A60BC
:1054640064E09DF81E300A2B03D09DF81E300D2BEE
:1054740006D13F20FDF70EF92E4B00221A6055E0AD
:105484009DF81E308DF81F3001F0D7FE03468DF8CD
:105494001E309DF81E303F2B03D1264B00221A608C
:1054A40044E09DF81E300D2B0ED09DF81F30DB001C
:1054B400DAB29DF81F305B00DBB21344DAB29DF818
:1054C4001E3013448DF81F309DF81F30013B8DF8BA
:1054D4001F309DF81F300F2B15D92020FDF7DAF867
:1054E4003120FDF7D7F82D20FDF7D4F83120FDF752
:1054F400D1F83620FDF7CEF82120FDF7CBF83F2078
:10550400FDF7C8F812E09DF81F309AB20A4B9A8052
:105514009DF81F309AB2094B9A80094B1B6843F4DB
:105524007F03074A1360034B00221A6009B030BDA1
:10553400046A0008A44100206C40002014400020AC
:045544009C41002066
:1055480000B583B01F4B01221A6001F0CEFC1E4843
:1055580001F0DCFF3A20FDF79BF82020FDF798F8D2
:1055680001F069FE03468DF807309DF807303F2BA0
:1055780003D1144B00221A6021E09DF807300A2B52
:1055880003D09DF807300D2B06D13F20FDF780F89A
:105598000C4B00221A6012E09DF807309AB20B4BB0
:1055A800DA809DF807309AB2094BDA80094B1B68FC
:1055B80043F47F03074A1360024B00221A6003B0CA
:1055C8005DF804FBA4410020AC7200086C40002088
:0855D800144000209C4100205A
:1055E00030B5BDB003468DF80730B04B35AC0FCBAE
:1055F00007C42380AE4B2FAC1D460FCD0FC495E8DA
:10560000030020600434218002340B0C2370A94B6A
:1056100025AC1D460FCD0FC40FCD0FC495E8030078
:10562000206004342170A44B15AC1D460FCD0FC46F
:105630000FCD0FC40FCD0FC495E80F0007C4237022
:105640009E4B0EAC1D460FCD0FC495E8070003C45A
:1056500022809B4B03AC1D460FCD0FC40FCD0FC452
:1056600095E8070003C42280964B01221A609DF83A
:1056700007305B005B00944A13443A939DF807306F
:105680005B005B00914A134439930023ADF8EC3082
:1056900001F02FFC35AB184601F03CFF01F0A9FCEE
:1056A0000346ADF8E230BDF8E230FF2B06D93F20CB
:1056B000FCF7F2FF834B00221A60B0E1BDF8E23044
:1056C000002B20D13A9B4FF6FF721A803A9B02338F
:1056D0004FF6FF721A80399B4FF6FF721A80399B82
:1056E00002334FF6FF721A809DF807301846FBF719
:1056F00031F8774B1B6843F47F03754A1360714B95
:1057000000221A608BE1BDF8E230F52B21D93A9BDB
:105710009A1C3A92BDF8E2201A803A9B80221A80A5
:10572000399B9A1C3992BDF8E2201A803A9B1A885C
:10573000399B1A809DF807301846FBF70BF8644B2D
:105740001B6843F47F03624A13605E4B00221A60B9
:1057500065E1BDF8E2300F2B04D8BDF8E2308DF8DA
:10576000EE3005E0BDF8E230DBB21B098DF8EE301B
:105770009DF8EE30082B06D83F20FCF78DFF514BEB
:1057800000221A604BE19DF8EE300D2B07D9BDF8D1
:10579000E230F22B03D0BDF8E230F32B6AD19DF852
:1057A000EE300C2B2CD09DF8EE300D2B28D0BDF810
:1057B000E230F32B24D02FAB184601F0ABFE454B63
:1057C0001B68002B03D0444801F0A4FE02E04348CC
:1057D00001F0A0FE3F20FCF75FFF2920FCF75CFFF3
:1057E0002020FCF759FF00F029F90346ADF8EC3012
:1057F000BDF8EC307F2B03D9324B00221A600EE14A
:1058000001F077FB9DF80730062B03D99DF8073090
:105810000B2B03D99DF807300E2B07D90EAB18467A
:1058200001F078FE00238DF8EF3092E025AB1846AA
:1058300001F070FE01F0DEFE03468DF8EF309DF8BA
:10584000EF300A2B0AD09DF8EF300D2B06D03F2009
:10585000FCF722FF1B4B00221A60E0E09DF8EF30BE
:105860000A2B03D180238DF8EF3072E000238DF8EE
:10587000EF306EE09DF8EE300E2B63D10023ADF8D3
:10588000EC309DF80730062B03D99DF807300B2B21
:1058900003D99DF807300E2B22D90EAB184601F024
:1058A00039FE00238DF8EF3053E000BF246A000872
:1058B000346A00084C6A0008746A0008B46A000878
:1058C000D06A0008A4410020784000202040002039
:1058D0009C410020904100204C670008446700086C
:1058E00001F007FB15AB184601F014FE01F082FE33
:1058F00003468DF8EF309DF8EF300A2B0ED09DF85F
:10590000EF300B2B0AD09DF8EF300D2B06D03F2047
:10591000FCF7C2FE434B00221A6080E09DF8EF3096
:105920000A2B03D180238DF8EF3012E09DF8EF3081
:105930000B2B03D181238DF8EF300AE000238DF883
:10594000EF3006E03F20FCF7A7FE364B00221A603E
:1059500065E09DF8EF30002B2DD101F0CAFA03ABC2
:10596000184601F0D7FD304B1B68002B03D02F48A1
:1059700001F0D0FD02E02E4801F0CCFD3F20FCF705
:105980008BFE2920FCF788FE2020FCF785FE00F026
:1059900055F803468DF8EF309DF9EF30002B03DB0F
:1059A0009DF8EF30002B06D13F20FCF775FE1D4B14
:1059B00000221A6033E09DF8EF301B021AB2BDF9E5
:1059C000EC3013431BB2ADF8EC303A9B9A1C3A9280
:1059D000BDF8E2201A803A9BBDF8EC201A80399B72
:1059E0009A1C3992BDF8E2201A803A9B1A88399B9A
:1059F0001A809DF807301846FAF7ACFE0D4B9B68ED
:105A000003F00103002B01D1FBF7C8FD0A4B1B6813
:105A100043F47F03084A1360024B00221A603DB032
:105A200030BD00BFA4410020904100204C67000819
:0C5A300044670008000004509C41002066
:105A3C0000B583B000238DF80730424B1B68002B58
:105A4C002FD0012001F083FB03468DF806309DF822
:105A5C000630EE2B01D1FF2370E09DF806308DF857
:105A6C000730012001F073FB03468DF806309DF8DA
:105A7C000630EE2B01D1FF2360E09DF80630FF2BA2
:105A8C0002D19DF8073059E09DF807301B015AB23E
:105A9C009DF9063013435BB28DF807309DF8073043
:105AAC004CE001F0C6FB03468DF806309DF806303D
:105ABC003F2B01D1FF2341E09DF806308DF80730D4
:105ACC0001F0B7FB03468DF806309DF806303F2BEE
:105ADC0001D1FF2332E09DF806300D2B02D19DF849
:105AEC0007302BE09DF807301A46920013445B00F8
:105AFC00DAB29DF8063013448DF8073001F099FBAB
:105B0C0003468DF806309DF806303F2B01D1FF235C
:105B1C0014E09DF806300D2B02D19DF807300DE0F6
:105B2C009DF807301A46920013445B00DAB29DF8D8
:105B3C00063013448DF807309DF80730184603B033
:085B4C005DF804FB904100200C
:105B540030B5DDB0884B56AC1D460FCD0FC495E86B
:105B6400030084E80300854B51AC1D460FCD0FC4E0
:105B74002B682380824A4FAB92E8030018600433F9
:105B84001970804B44AC1D460FCD0FC40FCD0FC40C
:105B940095E8070003C422800234130C23707A4B67
:105BA40034AC1D460FCD0FC40FCD0FC40FCD0FC4A1
:105BB40095E80F0007C4238002341B0C2370734A3A
:105BC40022AB11464622184601F077FB5CABA3F5E5
:105BD4009C736F4A184611464D231A4601F06DFB1B
:105BE4005CABA3F5B8736B4A1C4615460FCD0FC4C6
:105BF4000FCD0FC40FCD0FC495E80300206004340B
:105C0400217001F074F956AB184601F081FC01F0E3
:105C14006EF92120FCF73EFD3A20FCF73BFD2020E5
:105C2400FCF738FD51AB184601F072FC01F05FF946
:105C34005620FCF72FFD3A20FCF72CFD2020FCF722
:105C440029FD4FAB184601F063FC534801F060FC9A
:105C540001F04DF94220FCF71DFD3A20FCF71AFD36
:105C64002020FCF717FD4FAB184601F051FC4B48C0
:105C740001F04EFC01F03BF94D20FCF70BFD3A20FE
:105C8400FCF708FD2020FCF705FD4FAB184601F09A
:105C94003FFC434801F03CFC01F029F94320FCF7A8
:105CA400F9FC3A20FCF7F6FC2020FCF7F3FC4FABA0
:105CB400184601F02DFC3B4801F02AFC01F017F9CD
:105CC4004820FCF7E7FC3A20FCF7E4FC2020FCF732
:105CD400E1FC4FAB184601F01BFC334801F018FC03
:105CE40001F005F94420FCF7D5FC3A20FCF7D2FC7E
:105CF4002020FCF7CFFC4FAB184601F009FC2B48E1
:105D040001F006FC2A4801F003FC01F0F0F85820E9
:105D1400FCF7C0FC3A20FCF7BDFC2020FCF7BAFCE1
:105D24004FAB184601F0F4FB204801F0F1FB214889
:105D340001F0EEFB01F0DBF844AB184601F0E8FBA0
:105D440001F0D5F834AB184601F0E2FB01F0CFF8CE
:105D540022AB184601F0DCFB01F0C9F80EAB184683
:105D640001F0D6FB01F0C3F86B46184601F0D0FBF6
:105D740000BF5DB030BD00BFFC6A0008146B0008B2
:105D8400286B0008306B00085C6B00089C6B0008F3
:105D9400E46B0008346C00081C720008E866000814
:105DA40014670008D86E0008AC7200083867000851
:085DB400446700084C67000879
:105DBC0030B5BDB0A74B2FAC1D460FCD0FC40FCDCA
:105DCC000FC42B681A46228002341B0C2370A24B82
:105DDC0026AC1D460FCD0FC40FCD0FC42B682370FE
:105DEC009E4B20AC1D460FCD0FC495E803002060E0
:105DFC000434218002340B0C2370994B1BAC1D46D0
:105E0C000FCD0FC42B682370964A19AB92E8030090
:105E1C0083E80300944B12AC1D460FCD0FC495E8DC
:105E2C00070003C42270914B0BAC1D460FCD0FC461
:105E3C0095E8070003C422808D4A08AB07CA03C348
:105E4C001A708C4A05AB07CA03C31A808A4B01AC83
:105E5C000FCB84E80F0001F046F8884801F054FBA2
:105E6C0001F041F85620FCF711FC3A20FCF70EFC2F
:105E7C002020FCF70BFC19AB184601F045FB8048C1
:105E8C0001F042FB3A20FCF701FC2020FCF7FEFB62
:105E9C007C4B1A897B4B5B8913409BB24FF6FF728C
:105EAC00934204D140F28343ADF8EE300CE0754BD5
:105EBC001B891B021AB2734B5B891BB2DBB21BB280
:105ECC0013431BB2ADF8EE30BDF8EE30184601F0BE
:105EDC006DFA2F20FCF7DAFB2020FCF7D7FB694B7F
:105EEC009A89684BDB8913409BB24FF6FF72934241
:105EFC0004D145F24073ADF8EE300CE0614B9B8958
:105F0C001B021AB25F4BDB891BB2DBB21BB2134311
:105F1C001BB2ADF8EE30BDF8EE30184601F046FA83
:105F2C00594B1B6803F0FF23B3F57F4F2AD100F0C8
:105F3C00DAFF26AB184601F0E7FA544B1B891B021B
:105F4C001AB2524B5B891BB2DBB21BB213431BB2AE
:105F5C00ADF8EE30BDF8EE30184601F027FA4B4B99
:105F6C009B891B021AB2494BDB891BB2DBB21BB2F9
:105F7C0013431BB2ADF8EE30BDF8EE30184601F00D
:105F8C0015FA30E0404B1B6803F0FF23B3F1FF2FF1
:105F9C0029D100F0A8FF2FAB184601F0B5FA3B4B06
:105FAC001B891B021AB2394B5B891BB2DBB21BB2C9
:105FBC0013431BB2ADF8EE30BDF8EE30184601F0CD
:105FCC00F5F9324B9B891B021AB2304BDB891BB2A1
:105FDC00DBB21BB213431BB2ADF8EE30BDF8EE30A2
:105FEC00184601F0E3F900F07EFF4220FCF74EFB6F
:105FFC003A20FCF74BFB2020FCF748FB19AB18466A
:10600C0001F082FA224801F07FFA3A20FCF73EFBBD
:10601C002020FCF73BFB1B4B1B888DF8ED309DF8CB
:10602C00ED30184600F02EFA174B1B6823F47F0353
:10603C0023F47F43FF2B2DD100F055FF26AB1846E0
:10604C0001F062FA114B1B88DBB2184600F01AFA09
:10605C0035E000BF6C6C0008906C0008B46C000854
:10606C00CC6C0008E06C0008E86C0008046D0008BB
:10607C00206D00082C6D0008386D00085C7300085A
:10608C001C720008144000209C4100206C40002031
:10609C00E8660008AC4B1B6823F47F0323F47F43B2
:1060AC00AA4A93420BD100F01EFF2FAB184601F009
:1060BC002BFAA74B1B88DBB2184600F0E3F900F073
:1060CC0012FF4D20FCF7E2FA3A20FCF7DFFA202011
:1060DC00FCF7DCFA9F4801F017FA3A20FCF7D6FAE5
:1060EC002020FCF7D3FA9C4B5B884FF6FF7293424F
:1060FC0003D11F238DF8ED3003E0974B5B888DF8AF
:10610C00ED309DF8ED30184600F0BCF900F0EBFED8
:10611C004320FCF7BBFA3A20FCF7B8FA2020FCF736
:10612C00B5FA8E4801F0F0F93A20FCF7AFFA2020CE
:10613C00FCF7ACFA884B9B884FF6FF72934203D165
:10614C0001238DF8ED3005E0834B9B88DBB20133E6
:10615C008DF8ED309DF8ED309BB21846FCF7F8FA4F
:10616C0000F0C1FE4820FCF791FA3A20FCF78EFAB9
:10617C002020FCF78BFA7A4801F0C6F93A20FCF79C
:10618C0085FA2020FCF782FA734BDB884FF6FF72FE
:10619C00934203D102238DF8ED3003E06E4BDB8884
:1061AC008DF8ED309DF8ED303033DBB21846FCF74E
:1061BC006DFA00F098FE6B4801F0A6F96A4B1B686B
:1061CC00002B03D1694801F09FF902E0684801F007
:1061DC009BF900F088FE20AB184601F095F900F011
:1061EC0082FE01238DF8EC3040E19DF8EC305B0031
:1061FC005B00604A13443993399B02333893399BC3
:10620C001B880F2B12D8399B1B888DF8EA309DF810
:10621C00EA301B015BB223F00F035AB24E4B9B8842
:10622C005BB213435BB28DF8E9300CE0399B1B88F1
:10623C001B099BB2DBB203F00F038DF8EA30399BDC
:10624C001B888DF8E9309DF8EC305A1E1346DB00A4
:10625C009B1A5B00484A1344184601F055F9399BC8
:10626C001A88389B1B8813409BB24FF6FF729342DF
:10627C0003D1424801F048F9EDE01BAB184601F0A0
:10628C0043F99DF8E930184600F09DFD9DF8E93082
:10629C00F32B00F2CC809DF8E930F22B03D09DF863
:1062AC00EA300B2B39D8304B1B68002B14D0389BA1
:1062BC001B88DBB203F07F03DBB2184600F083FDD2
:1062CC00389B1B881B0A9BB2DBB203F07F03DBB24B
:1062DC00184600F078FD11E0389B1B8803F07F0313
:1062EC009BB21846FCF734FA389B1B881B0A9BB2EE
:1062FC0003F07F039BB21846FCF72AFA389B1B88E5
:10630C001BB2002B04DB0BAB184601F0FDF8A2E02E
:10631C0008AB184601F0F8F89DE09DF8EA300E2B1A
:10632C0059D1114B1B68002B2AD0389B1B88DBB230
:10633C00184600F048FD389B1B881B0A9BB2DBB249
:10634C00184600F040FD29E09C410020FF0000FFB2
:10635C006C4000201467000814400020D86E000820
:10636C00AC720008386700089041002044670008B0
:10637C004C67000820400020046F00086C73000874
:10638C00389B1B88DBB29BB21846FCF7E1F9389BB3
:10639C001B881B0A9BB21846FCF7DAF9389B1B8842
:1063AC0003F47F43B3F5014F04D105AB184601F05C
:1063BC00ABF850E0389B1B8803F47F43B3F5004FD8
:1063CC0004D108AB184601F09FF844E00BAB18461B
:1063DC0001F09AF83FE02A4B1B68002B08D0389B41
:1063EC001B881B0A9BB2DBB2184600F0ECFC06E0E3
:1063FC00389B1B881B0A9BB21846FCF7A9F9202076
:10640C00FCF744F92020FCF741F92020FCF73EF979
:10641C00389B1B881BB2002B04DB12AB184601F017
:10642C0073F818E008AB184601F06EF813E000237F
:10643C008DF8EB3007E02020FCF728F99DF8EB30C5
:10644C0001338DF8EB309DF8EB30062BF3D901AB13
:10645C00184601F059F89DF8EC30112B01D000F0E2
:10646C0042FD9DF8EC3001338DF8EC309DF8EC30AA
:10647C00112B7FF6BAAE00BF00BF3DB030BD00BFE0
:04648C00904100201B
:1064900000B583B003468DF807309DF80730644A95
:1064A000A2FB0323DB08DBB23033DBB21846FCF778
:1064B000F3F89DF807205E4BA3FB0213D9080B46A7
:1064C0009B000B445B00D31ADBB23033DBB21846BF
:1064D000FCF7E2F89DF80730602B00F08B80602B12
:1064E00000F39580262B41DC0B2BC0F290800B3BF8
:1064F0001B2B00F28C8001A252F823F07365000878
:106500000F6600080F6600080F6600080F66000897
:106510000F6600080F6600080F6600088D6500080A
:106520000F6600080F6600080F6600080F66000877
:106530000F6600080F6600080F6600080F66000867
:106540000F6600080F6600080F660008A7650008C0
:106550000F6600080F6600080F6600080F66000847
:106560000F6600080F660008C1650008392B34D09B
:106570004DE03520FCF790F83220FCF78DF8302004
:10658000FCF78AF83020FCF787F84DE03220FCF762
:1065900083F83020FCF780F83020FCF77DF82020CD
:1065A000FCF77AF840E04D20FCF776F84920FCF73C
:1065B00073F84420FCF770F84920FCF76DF833E0DD
:1065C0003420FCF769F83020FCF766F83020FCF73F
:1065D00063F82020FCF760F826E03620FCF75CF832
:1065E0003020FCF759F83020FCF756F82020FCF753
:1065F00053F819E03020FCF74FF83020FCF74CF846
:106600002020FCF749F82020FCF746F80CE03F205A
:10661000FCF742F83F20FCF73FF83F20FCF73CF83E
:106620002020FCF739F800BF00BF03B05DF804FB81
:04663000CDCCCCCC35
:10663400114B1B68104A43F0010313600E4B0022F8
:106644009A600D4B1B680C4A23F0A85323F41023C3
:106654001360094B4FF48052DA60074B1B68064AFB
:1066640023F480231360044B00229A61034B4FF000
:1066740000629A6000BF70470010024000ED00E025
:1066840082B001900A4B1B68002B0DDA084B1B6883
:10669400074A43F000431360019B18331A68019BB7
:1066A400183302321A6000E0FEE702B0704700BF00
:0466B4002CED00E0E9
:1066B80020286329323031362D323120572E53634A
:0866C80068656D6D65727400D8
:1066D00018035500530042002D004D00690064006E
:0866E000690043006F006D002A
:1066E80053657269616C20434F4D20426175647235
:1066F800617465202861637469766520696E20522B
:0C670800532D323332204D6F64652900A0
:106714004D49444920426175647261746520286161
:10672400637469766520696E204D494449204D6F34
:04673400646529006F
:0C6738004E756D626572426173653D0034
:08674400646563696D616C007E
:04674C006865780004
:10675000FEE7FEE7FEE7FEE7FEE7FEE7FEE7FEE711
:10676000FEE7FEE7FEE7FEE7FEE7FEE7FEE7FEE701
:10677000FEE7FEE7FEE7FEE7FEE7FEE7FEE7FEE7F1
:10678000FEE7FEE7FEE7FEE7FEE7FEE7FEE7FEE7E1
:10679000FEE7FEE7FEE7FEE7FEE7FEE7FEE7FEE7D1
:1067A000FEE7FEE7FEE7FEE7FEE7FEE7FEE7FEE7C1
:1067B000FEE7FEE7FEE7FEE7FEE7FEE7FEE7FEE7B1
:1067C000FEE7FEE7FEE7FEE7FEE7FEE7FEE7FEE7A1
:1067D000FEE7FEE7FEE7FEE7FEE7FEE7FEE7FEE791
:1067E000FEE7FEE7FEE7FEE7FEE7FEE7FEE7FEE781
:1067F000FEE7FEE7FEE7FEE7FEE7FEE7FEE7FEE771
:10680000FEE7FEE7FEE703488546FFF713FF00F0CB
:0868100003B87047008001206D
:1068180011488546114C20680434004201D0804755
:10682800F9E70F480F49091A082903DB002202601B
:10683800043001600C480D49884205D002680430D4
:1068480003B4904703BCF7E700208646EC460020D7
:106858000021074A9047FEE7008001201C760008C7
:10686800C8410020C8450020597100085971000826
:046878004D020008C5
:10687C001EF0040F0CBFEFF30880EFF30980014901
:08688C000847000085660008C2
:10689400536574757020686173206368616E676501
:1068A400642E2053617665207769746820277C27DD
:1068B40020666F72207065726D616E656E742073F0
:1068C400746F7261676520696E20466C617368003D
:1068D4002020202020202043616E63656C204578B1
:1068E40069742077697468203C4553433E00000076
:1068F4005361766520746F20466C6173683F202D68
:106904003E7479706520616761696E200000000043
:10691400204E4F542053415645442120000000008E
:106924002052656C6F6164205365747570206672C3
:106934006F6D20466C6173683F202D3E74797065DD
:1069440020616761696E2000204E4F542052454CEF
:106954004F41444544212000436F6E6669672049D6
:106964006E7075742320000020656E746572206E4D
:1069740065772056696420283420686578206E691C
:1069840062626C6573293A200000000020656E7411
:106994006572206E6577205069642028342068650C
:1069A40078206E6962626C6573293A2000000000E9
:1069B400434F4D20626175642072617465202D20FF
:1069C400656E74657220666972737420322064691E
:1069D400676974733A2000004D4944492062617527
:1069E400642072617465202D20656E746572206662
:1069F400697273742032206469676974733A200081
:106A0400456E746572204D494449206368616E6E19
:106A1400656C2028312E2E2E3136293A20000000B4
:106A240053746174757328686578293F20000000E9
:106A3400202D3E317374204D4944492064617461B2
:106A440020627974652800002020506F72742052EF
:106A54006561643A2744273D6469676974616C2CF5
:106A64002741273D616E616C6F673F200000000085
:106A74002020506F727420526561643A2744273D88
:106A84006469676974616C2C2741273D616E616C90
:106A94006F672837626974292C2742273D616E612C
:106AA4006C6F67283132626974293F20000000004E
:106AB4002020506F727420526561643A20646967C3
:106AC4006974616C206F6E6C7900000020206C6129
:106AD4007374204D4944492064617461206279745F
:106AE40065207768656E20627574746F6E207075AA
:106AF40073686564280000004C697374206F662015
:106B0400536574757020436F6D6D616E64733A00E4
:106B14006C6973742041637475616C20536574757A
:106B2400700000007365742000000000312C322CCA
:106B3400332C342C352C362C372C382C392C313042
:106B44002C31312C31322C31332C31342C312C3149
:106B54002C31362C553A0000202020736574204DCA
:106B6400494449206D7367732072656C6561736570
:106B740064206279206368616E6765206F662049CE
:106B84002F4F206E6F20312E2E39202B55736572B6
:106B9400427574746F6E0000403A2072656C6F61C8
:106BA400642073657475702066726F6D20466C6125
:106BB400736820286368616E6765732073696E6308
:106BC40065206C61737420506F7765725570206115
:106BD40072652063616E63656C6C656429000000F6
:106BE4007C3A2073617665206E65772073657475D1
:106BF40070207065726D616E656E746C7920696E5B
:106C040020466C617368202877696C6C2062656328
:106C14006F6D6520616374697665206174206E65AB
:106C2400787420506F776572205570290000000039
:106C3400453A20657869742053455455502C207288
:106C4400657475726E20746F20626964697265631D
:106C540074696F6E616C20636F6D6D756E696361CD
:106C640074696F6E0000000020202020202028730B
:106C7400617665642C206E6F74207965742061637D
:106C8400746976652C206E65773A000020202020F8
:106C94002020286D6F6469666965642C206E6F74AA
:106CA4002073617665642C206E65773A00000000DD
:106CB400496E707574204368616E6765206D6573F5
:106CC40073616765733A000020636F6E6669677568
:106CD400726564206D736720000000004163747561
:106CE400616C2000204469673A73656E64206461B6
:106CF4007461206966207075736865640000000023
:106D0400204469673A73656E64206461746132205B
:106D140069662070757368656400000020416E61C7
:106D2400376269740000000020416E61313262698B
:106D34007400000053696E676C6520627974652085
:046D44006D73670004
:0E6D48005553422D4D696469436F6D207600EE
:106D560000B583B00123019305E00198F9F7F7FC2C
:106D6600019B01330193019B112BF6D900BF00BF94
:066D760003B05DF804FB10
:106D7C00120110010200004083044057060300007A
:026D8C00000104
:106D8E0000B585B003468DF807309DF807303033D7
:106D9E008DF80F309DF80F30392B04D99DF80F3038
:106DAE0007338DF80F309DF80F301846FBF7F1FBC7
:106DBE009DF807301846FBF752FC00BF05B05DF892
:026DCE0004FBC4
:026DD0000000C1
:106DD20000B585B003468DF807309DF807301B09D2
:106DE2008DF80F309DF80F3030338DF80F309DF84D
:106DF2000F30392B04D99DF80F3007338DF80F303F
:106E02009DF80F301846FBF746FC9DF8073003F05B
:106E12000F038DF80F309DF80F3030338DF80F309F
:106E22009DF80F30392B04D99DF80F3007338DF8B8
:106E32000F309DF80F301846FBF72DFC2020FBF792
:0A6E42002AFC00BF05B05DF804FB58
:106E4C0012010002000000408304425706030001B7
:026E5C00000133
:106E5E0000B585B00346ADF80630BDF80630B3F583
:106E6E00805F03D340F6FF73ADF80630BDF80630F1
:106E7E001B0A9BB2DBB203F00F038DF80F309DF8A7
:106E8E000F301846FBF72BFCBDF806301B099BB2E2
:106E9E00DBB203F00F038DF80F309DF80F3018465C
:106EAE00FBF71DFCBDF80630DBB203F00F038DF8C7
:106EBE000F309DF80F301846FBF711FC2020FBF722
:0A6ECE00E4FB00BF05B05DF804FB13
:106ED800476C6F62616C204D494449204368616E7C
:0A6EE8006E656C28312D313629004B
:106EF20008B50D20FBF7CFFB0A20FBF7CCFB00BF48
:026F020008BDC8
:106F0400496E707574312028504132293A00496E17
:106F1400707574322028504133293A00496E7075D7
:106F240074332028504230293A00496E7075743405
:106F34002028504134293A00496E70757435202850
:106F4400504131293A00496E7075743620285041F9
:106F540030293A00496E707574372850413135290B
:106F64003A00496E707574382028504237293A0027
:106F7400496E707574392028504233293A00496E9D
:106F8400707574313028504235293A00496E707555
:106F940074313128504234293A00496E7075743185
:106FA4003228504137293A00496E707574313328BC
:106FB400504136293A00496E707574313428504175
:106FC40035293A00496E7075743135285042392993
:106FD4003A00496E707574313628504238293A00A7
:0E6FE400496E707574552850433133293A00B8
:106FF20000B583B00023ADF80630012000F0ACF8F4
:1070020003468DF805309DF80530ED2B02D94FF47B
:107012007F436AE09DF805309BB21B01ADF8063054
:10702200012000F099F803468DF805309DF80530EF
:10703200EE2B02D14FF47F4357E09DF80530FF2B32
:1070420019D1BDF80630002B02D1BDF806304CE054
:10705200BDF806301B09ADF80630BDF80630082B26
:1070620003D9BDF806300E2B02D94FF47F433CE022
:10707200BDF8063039E09DF805309AB2BDF8063009
:107082001343ADF80630BDF80630002B02D1BDF82F
:1070920006302AE0BDF806308F2B02D84FF47F432A
:1070A20023E0BDF80630F02B03D0BDF80630F72BF5
:1070B20002D14FF47F4318E0BDF80630F12B0FD018
:1070C200BDF80630F42B0BD0BDF80630F52B07D0F7
:1070D200BDF80630F92B03D0BDF80630FD2B02D1E6
:1070E2004FF47F4301E0BDF80630184603B05DF867
:0270F20004FB9D
:1070F4000902650002010080310904000000010159
:107104000000092401000109000101090401000231
:1071140001030000072401000141000624020101CB
:1071240000062402020200092403010301020100F3
:107134000924030204010101000905810240000041
:1071440000000525010103090502024000000000BA
:05715400052501010109
:10715A0000B585B003468DF8073000BFFBF7F7FB93
:10716A000346ADF80C30BDF80C30002BF6D0BDF854
:10717A000C308DF80F309DF80730002B09D09DF8A0
:10718A000F300A2B03D09DF80F300D2B01D1FF23AE
:10719A003BE09DF80F303F2B04D13F20FBF777FAF5
:1071AA00EE2332E09DF80F30602B08D99DF80F309E
:1071BA007A2B04D89DF80F30203B8DF80F309DF8BC
:1071CA000F30402B08D99DF80F30462B04D89DF874
:1071DA000F30073B8DF80F309DF80F302F2B10D949
:1071EA009DF80F303F2B0CD89DF80F30303B8DF8AF
:1071FA000F309DF80F301846FBF773FA9DF80F30E1
:10720A0003E03F20FBF743FAEE23184605B05DF88A
:02721A0004FB73
:10721C00555342205669642F506964206F66207460
:10722C0068697320646576696365202868657829C8
:01723C000051
:10723E0000B583B000BFFBF788FB0346ADF8063000
:10724E00BDF80630002BF6D0BDF806308DF80530AF
:10725E009DF805300A2B03D09DF805300D2B01D17A
:10726E000D2318E09DF805302F2B03D99DF805301E
:10727E00392B04D93F20FBF708FA3F230BE09DF88A
:10728E0005301846FBF701FA9DF80530303B8DF8B6
:0E729E0005309DF80530184603B05DF804FB7E
:1072AC004879737465726573697328302E2E392989
:0172BC0000D1
:1072BE00844640EA010313F0030F18D18446202AB6
:1072CE000BD32DE9F007B1E8F807A0E8F807A2F113
:1072DE002002202AF7D2BDE8F007042A07D351F87E
:1072EE00043B40F8043BA2F10402042AF7D2002A20
:1072FE0005D011F8013B00F8013B013AF9D1604687
:02730E007047C6
:107310000902430002010080310904000001020259
:1073200000000524001001052401030004240207C5
:10733000052406000107058303100040090401002D
:10734000020A000000070581024000010705020251
:03735000400001F9
:0773540000C2010000000867
:0F735C00436F6E66696775726174696F6E3A0090
:10736C00204E4F206D736720636F6E666967757270
:03737C0065640045
:077380004572726F723A00C2
:1073880000B583B003468DF807309DF807301846DE
:10739800FBF702F99DF807301846FBF763F99DF8EB
:1073A80007301846FCF74AFF00BF03B05DF804FB3E
:1073B80000B585B00346ADF80630BDF806301B0BA6
:1073C8009BB2DBB203F00F038DF80F309DF80F303E
:1073D8001846FBF787F9BDF806301B0A9BB2DBB2EB
:1073E80003F00F038DF80F309DF80F301846FBF7A8
:1073F80079F9BDF806301B099BB2DBB203F00F0325
:107408008DF80F309DF80F301846FBF76BF9BDF873
:107418000630DBB203F00F038DF80F309DF80F3004
:107428001846FBF75FF92020FBF732F900BF05B0DB
:047438005DF804FBFC
:10743C0000B585B00190019B1B0FDBB203F00F036D
:10744C008DF80F309DF80F301846FFF79AFC019B12
:10745C001B0EDBB203F00F038DF80F309DF80F30CD
:10746C001846FFF78EFC019B1B0DDBB203F00F03DC
:10747C008DF80F309DF80F301846FFF782FC019BFA
:10748C001B0CDBB203F00F038DF80F309DF80F309F
:10749C001846FFF776FC019B1B0BDBB203F00F03C6
:1074AC008DF80F309DF80F301846FFF76AFC019BE2
:1074BC001B0ADBB203F00F038DF80F309DF80F3071
:1074CC001846FFF75EFC019B1B09DBB203F00F03B0
:1074DC008DF80F309DF80F301846FFF752FC019BCA
:1074EC00DBB203F00F038DF80F309DF80F30184608
:1074FC00FFF747FC2020FBF74DF82020FBF7B0F8F6
:08750C0000BF05B05DF804FBAF
:1075140000B585B0019004E09DF80F301846FBF7E4
:10752400B9F8019B5A1C01921B788DF80F309DF815
:107534000F30002BF0D100BF00BF05B05DF804FB95
:1075440000B583B04FF0A0435A694FF0A0439B6944
:1075540013400193019B002B46D0019B03F40023AD
:10756400002B01D0FCF7CAF8019B03F48023002B05
:1075740001D0FBF7FFFE019B03F01003002B01D0A9
:10758400FBF79EFD019B03F00803002B03D04FF093
:10759400A04308225A61019B03F48053002B06D0B8
:1075A400FBF72EFC4FF0A0434FF480525A61019B2D
:1075B40003F40053002B04D04FF0A0434FF40052C7
:1075C4005A61019B002B04DA4FF0A0434FF00042B4
:1075D4005A61019B03F40063002B06D04FF0A043D3
:1075E4004FF400625A6100E000BF03B05DF804FB91
:1075F40000B583B00120FFF7AEFD03468DF80730D8
:107604009DF80730EE2B01D1FF2301E09DF80730F0
:08761400184603B05DF804FB09
:10761C005176000814000020B34100006776000882
:10762C00000000203C760008140000000000000060
:10763C0012100020122000201230002012400020D6
:04764C0000093D00F4
:10765000206861680834094204D0002202700130B9
:067660000139FBD1704767
:1076660020686168A2680C34124205D00B7803705A
:0A76760001300131013AF9D17047EB
:040000050800680780
:00000001FF
